:1080000000000120051301005DEA00005DEA0000A8
:108010005DEA00005DEA00005DEA0000000000008B
:108020000000000000000000000000005DEA000009
:108030005DEA0000000000005DEA00001D8600000F
:108040005DEA00005DEA00005DEA00005DEA000014
:108050005DEA00005DEA00005DEA00005DEA000004
:108060005DEA00005DEA00005DEA00005DEA0000F4
:108070005DEA00005DEA00005DEA00005DEA0000E4
:108080005DEA00005DEA00005DEA00005DEA0000D4
:108090005DEA00005DEA00005DEA00005DEA0000C4
:1080A0005DEA0000A5DA00005DEA00005DEA00007C
:1080B0005DEA00005DEA00005DEA00005DEA0000A4
:1080C0005DEA00005DEA00005DEA00005DEA000094
:1080D0005DEA00005DEA00005DEA0000B9D600003C
:1080E0005DEA00005DEA00005DEA00005DEA000074
:1080F0005DEA00005DEA00005DEA00005DEA000064
:108100005DEA00005DEA00005DEA00005DEA000053
:108110005DEA000079FC00005DEA00005DEA000015
:108120005DEA00005DEA00005DEA00005DEA000033
:108130005DEA00005DEA00005DEA00005DEA000023
:108140005DEA00005DEA0000718700005DEA000062
:108150005DEA00005DEA00005DEA00005DEA000003
:108160005DEA0000F5D600005DEA00005DEA00006F
:108170005DEA00005DEA00005DEA00005DEA0000E3
:088180005DEA00005DEA000069
:10840000FFFFFFFFFFFFFFFFFFFFFFFF7EF9FFFF03
:1084100010B5054C237833B9044B13B10448AFF3BE
:1084200000800123237010BD0086FF1F00000000A4
:10843000641801000C4B43B10C480D4910B5AFF363
:1084400000800C48036823B910BD0A48036833B99B
:108450007047094B002BF7D0BDE810401847064B7A
:10846000002BF5D0184700BF000000006418010081
:108470000486FF1F7485FF1F0000000080F3118831
:1084800070472F4B41F238015A5842F478525A50F3
:108490002C4A927902F00C020C2A4FD041F244028D
:1084A0002949995003F558339A78110748BF9A78AB
:1084B000264944BF42F008029A70214B41F244021F
:1084C000995041F204015A5842F4803242F0C002FD
:1084D0005A501A6842F440221A6003F5E833242205
:1084E0005A701B4A80211170A2221A70DA7802F0A9
:1084F0001F02DA7003221A7100225A719A799207C8
:10850000FCD59A79D006FCD40E4B19469A7902F024
:108510000C02082AFAD140225A718B7903F00C031D
:10852000082BFAD1074B1A4699794906FCD5222126
:108530001970937903F00C030C2BFAD1704700BF2C
:1085400000700440004006400000330100001301A9
:10855000005006402B4B5A7902F0E0025A711A790A
:1085600002F0F8021A71284A136843F004031360FA
:10857000264A136823F0784323F001031360244B49
:108580001A7802F08C0242F050021A705A7802F007
:108590009C0242F040025A709A7802F0E6029A7009
:1085A0001C4A0023137083F311881B4B012283F8AC
:1085B000182383F81923022283F83C2383F83D23F0
:1085C00083F84B2383F84C2383F84D2383F84E2301
:1085D00083F84F23032283F81F2383F8212383F892
:1085E000232383F8252383F84223042283F82723B7
:1085F000052283F84923062283F83B23072283F8C8
:108600003523704700F007404080044000D0004010
:1086100000D0074000E0074000E100E00C4A13688A
:10862000013313600B4A1368013313600A4B1A6855
:108630003AB11A68013A1A601B6813B9074B012254
:108640001A70074B1A6812B11A68013A1A6070471B
:108650001C86FF1F8497FF1F1C93FF1F1893FF1F8B
:108660002093FF1F024B034A5A6007221A6070478B
:1086700010E000E000770100014B1868704700BF70
:108680001C86FF1F1449154B41F22802072888BF9A
:10869000002010B553F82030114CB4FBF3F48B5884
:1086A00043F480638B500F4B4FF440729A63422027
:1086B000DA6306F0F1F90C4B0022DA709A709A71C5
:1086C000DA725A71C4F30422E4B21A705C70DA7878
:1086D00042F02C02DA7010BD00700440B0150100A9
:1086E000C0C62D0000B0044000A00E40094A136827
:1086F00051680133202B08BF00238B4208D011683A
:10870000114408721360044AD37843F08003D37095
:10871000704700BF2086FF1F00A00E400A4B996AD9
:10872000DA6A91420DD09A6A511C1A44996292F801
:10873000302002709A6A202A01D100229A62012018
:1087400070470020704700BF2086FF1F044B1A7837
:1087500002F0FF0012B100221A700120704700BF22
:108760001893FF1F014B1865704700BF2086FF1F3D
:1087700030B526480179C9B28C0617D5244BDA6A80
:108780009C6A0132202A08BF0022A2421BBFDC6A79
:10879000C579C27918191EBFEDB280F83050DA627F
:1087A0001C4A052010601A6D1B4B1A604A0608D53A
:1087B0001A4B4FF480529A60144AD37803F0BF03E7
:1087C000D3700B061BD5144B1868C0B9104B196831
:1087D0005A68914214D0114A4FF4805151605A683E
:1087E000511C1A445960117A084AC9B2D1715968AA
:1087F000202908BF5860D37843F04003D37030BDC0
:10880000024AD37803F07F03F8E700BF00A00E40D0
:108810002086FF1F1C93FF1F2093FF1F80F00F4037
:1088200062B67047FFF7FCBF72B67047FFF7FCBF38
:108830004FF0E02318B1034AC3F80C2D7047024AE9
:10884000FAE700BF0400FA050100FA05F7B5464C47
:108850004649474D474E4FF4807306226360A3603C
:1088600023618A6010224A601E224A61424A536292
:108870009364D3644FF400226A61AA603F4A4FF4C4
:10888000907050621363936402F5342280324FF487
:10889000905090604FF48020506000F590505061EF
:1088A000374A40F20310106050609060D060106151
:1088B00050619061D06133480022426132480361C7
:1088C00043618361836600F5322000F58070866025
:1088D0004661082623601046E360B4460A242B460E
:1088E00017468E46C1F804C00197019DB5F57A7F01
:1088F00030D3DEF810508E60ED0748BF013001978D
:10890000019DB5F57A7F29D3DEF81050ED0758BFE9
:108910000132013CE6D10A281C4923D10A2A21D17F
:1089200001220A70104A4FF4E0611160D16002F533
:108930003622102191604FF400225A600E4A4FF403
:108940008071116001225A605A6942F001025A6135
:1089500003B0F0BD019D01350195C6E7019D0135CC
:108960000195CDE70022DCE70090044000F00F40C5
:1089700040F00F407000000400A0044000B004402C
:1089800000C00440C0F00F4000D004407093FF1FAF
:10899000F7B5104B1B78D3B10F4B104D02210F468A
:1089A000042000241E469F6058600194019AAA4248
:1089B00009D97160B0600194019AAA42F3D8019A72
:1089C00001320192F8E7019A01320192EEE703B019
:1089D000F0BD00BF7093FF1F00F00F401FA1070004
:1089E000032806D8DFE800F00206080A1022054B2B
:1089F0005A6070472022FAE74022F8E74FF0806281
:108A0000F5E700BF00F10F40032806D8DFE800F0CB
:108A10000206080A1022054B9A6070472022FAE7E6
:108A20004022F8E74FF08062F5E700BF00F10F4009
:108A300010B50021044644FA01F3DB07C8B205D59E
:108A4000FFF7CEFF01310829F5D110BDFFF7DCFF9C
:108A5000F8E708B5032813D8DFE800F0020C0E1081
:108A6000002004F0ADFE43F27C03984294BF002046
:108A7000012008BD0120F4E70220F2E70320F0E71F
:108A8000002008BD032817D8DFE800F002070C110A
:108A90000A4B1868C0F300107047084B1868C0F301
:108AA00040107047054B1868C0F380107047034BA7
:108AB0001868C0F3806070470020704700F10F40D5
:108AC00070B5002425460126E0B2FFF7C2FF18B1B9
:108AD00006FA04F31D43EDB20134082CF4D1284604
:108AE00070BD024B1869C043C0B27047C0F00F4060
:108AF00037B50446FFF7C0FD0546FFF7BDFD401B37
:108B00000028B8BF40420128F7DD0020012C8DF875
:108B100004008DF8050010D007D3022C11D00306F5
:108B200048BF60F0FF0003B030BD022201A99020D1
:108B300005F074F89DF80400F1E7022201A99220E3
:108B4000F6E7224601A99420F2E708B5082004F0D0
:108B500037FE5E280ED9104B1A780AB901221A7016
:108B6000082004F02DFEA9280CD90C4B4FF40072FC
:108B70005A6008BD082004F023FE5428F0D80022D3
:108B8000054BECE7082004F01BFE95289EBF034B25
:108B90004FF400729A6008BD7486FF1F80F00F408A
:108BA000034B1878013801288CBF00200120704742
:108BB0007486FF1F034B1878012806BF02221A7023
:108BC000002070477486FF1FC0B205F035BDC0B2EB
:108BD00005F020BD08B507F073FE06F031F906F088
:108BE000E1F8BDE8084007F0EDBE38B5054606F0EF
:108BF0002FF808280AD900242819013406F0A8F80B
:108C0000092CF9D106F0D8F8012038BD002038BD74
:108C1000092106F03DB8002006F0CABA22492348CF
:108C200041F23C028B5843F440538B50204B0121BE
:108C300019601A6802431A601E4ADA601A61DA6A19
:108C400042F08052DA621A6822F001021A601A6851
:108C500022F000621A60184A4FF4007313605360E8
:108C60009360D360136153619361D361A2F5F032D5
:108C700011601168014311601049D16001F52001B4
:108C80001161D16A41F08051D162116821F0010176
:108C90001160116821F00061116002F5E832936201
:108CA000D36213645364704700700440000C1F804B
:108CB00000C002400300013E00B004400400513EE9
:108CC000FF2810B54FEA004323D82B4C03F47C1344
:108CD0008AB141F000610B436363E36A002BFCDA65
:108CE000254BDA6AD000FCD5986BDA6A42F0104264
:108CF000C0B2DA6210BD41F000410B436363E36A26
:108D0000002BFCDAA06BE36A43F01043C0B2E362CD
:108D100010BDB0F5007F17D2184C03F47C135AB184
:108D200041F000610B436363E36A002BFCDA134BF1
:108D3000DA6AD100FCD5D7E741F000410B43636309
:108D4000E36A002BFCDADDE70D4C03F47C135AB127
:108D500041F000610B436363E36A002BFCDA084BCC
:108D6000DA6AD200FCD5BFE741F000410B436363F0
:108D7000E36A002BFCDAC5E700C0024000D00240E5
:108D800000C00A4010B5FFF777FC0446FFF774FCFB
:108D9000001B0028B8BF40420628F7DD10BD07B50C
:108DA000030A8DF805008DF80610032201A9A02002
:108DB0008DF8043004F00CFFFFF7E4FF03B05DF81A
:108DC00004FBF0B5154600228BB00F461446AC42AA
:108DD00001D10BB0F0BD0AAB1344395D03F8221C7E
:108DE000531CC618F10602D0691E8C420DD1030A2D
:108DF0008DF80500033201A9A0208DF8043004F09D
:108E0000E7FEFFF7BFFF3046002301341A46DEE7D6
:108E10001FB5030A8DF80C30022203AB8DF80D004C
:108E200000921946A02004F01FFF9DF80C0005B029
:108E30005DF804FB1FB5030A8DF80C308DF80D00AA
:108E400000920B46022203A9A02004F00DFF05B0FA
:108E50005DF804FBC0EBC000072200F5B040FFF74F
:108E6000B0BFC0EBC000072200F5B040FFF7E2BF83
:108E700030B500238BB001AD1A465A550133222B71
:108E8000FBD14FF4B044230A8DF805402222294635
:108E9000A02020348DF8043004F09AFEFFF772FF12
:108EA000B4F5803FEFD10BB030BD13B50C46C0EB2D
:108EB000C0000722694600F5B040FFF7BBFF9DF8F0
:108EC000002023789A4212D19DF8012063789A42BB
:108ED0000DD19DF80220A3789A4208D1DDF8030055
:108EE000D4F80330C31A5842584102B010BD0020D4
:108EF000FBE77047F7B545F2FF70FFF789FF55288C
:108F000003D1354B1B78002B43D0002145F2FF7075
:108F1000FFF745FFFFF7ACFF40223049304F314E9D
:108F20000020FFF74EFF4FF4B76540242046402253
:108F30003946FFF746FF4034284660223146FFF7A6
:108F400040FFB4F5807F05F16005EFD102AD00234D
:108F500045F8043D4FF4D36440F6780620460422D9
:108F600029460434FFF72DFFB442F7D100230193C3
:108F70004FF4FF6440F6D806204604222946043404
:108F8000FFF71FFFB442F7D1552145F2FF70FFF7FD
:108F900006FF40221149144D124E0020FFF74AFFF0
:108FA000402210461149FFF745FF4022104980201A
:108FB000FFF740FF40220F49C020FFF73BFF00248E
:108FC000281960223146603407F010FDB4F5907F17
:108FD000F6D103B0F0BD00BF7093FF1F0C80FF1FE0
:108FE00040160100E0150100C494FF1F9493FF1F79
:108FF000F893FF1F5C94FF1F044B9B78022B044BDC
:109000008CBF042203221A70704700BF6C96FF1FAA
:109010008897FF1F38B5044CA0786378022807D9D9
:10902000024B04221A7038BD6C96FF1F8897FF1FF1
:10903000FF2B00F28784DFE813F0D301E701FB0187
:10904000050210021A0222022A0232024F025402C0
:109050005C02640277028A0292029C02A402AC02C1
:10906000B602BE02C802D002D602DC02E202E80268
:10907000EE02F40207038504850485040F0315033B
:109080008504850485048504850485048504850498
:1090900085048504850485048504850485041B03F3
:1090A0008504850485048504850485048504850478
:1090B0008504850485048504850485048504850468
:1090C0008504850485048504850485048504850458
:1090D0008504850485048504850485048504850448
:1090E0008504850485048504850485048504850438
:1090F0008504850485048504850485048504850428
:109100008504850485048504850485048504850417
:109110008504200328033003380340034803500329
:109120005803600368037003780380038803850491
:1091300099039F03A703AF03B703BD03C3038504CC
:10914000CA03D003D603DB038504E303EC03F50372
:109150008504FD0385048504850485048504850450
:1091600085048504850485048504850485048504B7
:10917000850485048504850485048504850400012F
:10918000140119011E012C013A013F01440149015A
:109190004E01530158015D01850485046201850477
:1091A00067016C018504710185048D0192019701AD
:1091B000B301B801BD01C3018504850407040F0490
:1091C0001A0426042C048504850432043A043F045E
:1091D0008504CE018504470485044D0452045D04D2
:1091E000850465046D04750485048504850485047F
:1091F0008504850485048504850485048504850427
:109200008504850485048504850485048504850416
:109210008504850485048504850485048504850406
:1092200085048504850485048504850485048504F6
:1092300085048504850485047D0405F002F89C4BB3
:1092400058609C4B1B785BB1994B5A689A4B1A60DB
:109250009A4B002A40F07A831A6842F008021A609A
:1092600038BD05F018F8924B5860EAE705F021F890
:109270008F4B5860E5E705F00EF88D4D20B9A078CA
:1092800005F031F86860DCE7A07805F019F868604F
:10929000D7E705F000F8864D20B9A07804F0CAFFA2
:1092A0006860CEE7A07805F017F86860C9E704F0B9
:1092B000AFFF7F4B5860C4E705F0C0F87C4B5860A7
:1092C000BFE705F09BF87A4B5860BAE705F09DF8C8
:1092D000774B5860B5E705F08AF8754B5860B0E7F2
:1092E00005F09AF8724B5860ABE705F0AEF8704B9A
:1092F0005860A6E705F097F86D4B5860A1E704F0B9
:10930000B5FF6B4B58609CE704F0EFFF684B58606B
:1093100097E76B4B1A5C664B5A6092E7142104F096
:1093200025FE634D674A0028D5BF6FF07F43664B2B
:109330006B6093FBF0F0A378C8BF6860642101FB09
:1093400003231B7E002B7FF47CAF686805F07DFB58
:10935000686076E704F0A6FF554B586071E704F0AB
:1093600077FF534B58606CE7132104F0FFFD504D1D
:10937000544A0028D5BF6FF07F43534B6B6093FB7B
:10938000F0F0A378C8BF6860642101FB03231B7E53
:10939000002B7FF456AF686805F057FB686050E714
:1093A00005F0DEF8424B58604BE705F0E0F8404B23
:1093B000586046E7712104F0D9FD3D4B586040E705
:1093C000002104F0D3FD10F0040F394B14BF01222B
:1093D00000225A6035E705F0A7F8354B586030E7B2
:1093E00003F020FB324D372120B9A07805F084F935
:1093F000686026E7A07805F07FF9A278334B53F830
:109400002230C01A68601CE760234343304A284D6D
:10941000D35C21211BB905F06FF9686011E705F0F5
:109420006BF9A278294B53F82230C01A686008E71C
:10943000284B242153F8204005F05EF9A0471C4B2F
:109440005860FEE6234B222153F8204005F054F9E2
:109450000002A047164B5860F3E61E4B03EB800258
:1094600053F82030D0689847114B5860E9E6154A08
:10947000642303FB00200E4B826A5A60E1E6114A26
:10948000642303FB00200A4B427A5A60D9E60D4A56
:10949000642303FB0020064B827A5A60D1E60F2139
:1094A00005F02AF9024B00F001005860C9E600BF40
:1094B0008897FF1F8397FF1F7497FF1F7496FF1FE6
:1094C0004C93FF1F9493FF1F0024F4004093FF1F51
:1094D000C494FF1F7886FF1F05F0B0FA9F4B5860B9
:1094E000AFE60F2105F008F99C4BC0F3002058604F
:1094F000A7E60F2105F000F9984BC0F3C0105860A3
:109500009FE6012105F0F8F8830741BF934A5368AD
:1095100043F00103536005077FF593AE8F4A53680C
:1095200043F0020353608CE6012105F0E5F8C4071F
:1095300041BF8A4A536843F00103536041077FF5F6
:1095400080AE864A536843F00203536079E6844A4A
:10955000642303FB0020814BC27D5A6071E6814B7E
:10956000252153F8204005F0C7F8A0477B4B5860F1
:1095700067E67B4A642303FB0020784B026B5A604A
:109580005FE6774A642303FB0020744BC26A5A608B
:1095900057E6744B272153F8204005F0ADF8A0475B
:1095A0006E4B58604DE66E4A642303FB00206B4B04
:1095B000426B5A6045E66B4B262153F8204005F07C
:1095C0009BF8A047654B58603BE6654A642303FB64
:1095D0000020624B826B5A6033E62D2105F08CF837
:1095E0005E4B58602DE62E2105F086F85B4B5860E7
:1095F00027E62F2105F080F8584B586021E63021EE
:1096000005F07AF8554B58601BE6332105F074F8E5
:10961000524B586015E6342105F06EF84F4B5860F8
:109620000FE6012105F068F8420641BF4B4A536836
:1096300043F00103536003067FF503AE474A5368C6
:1096400043F002035360FCE5012105F055F8434B5C
:10965000C0F301205860F4E5012105F04DF810F049
:10966000100FB2E6012105F047F810F0200FACE62C
:1096700003F060FD394B5860E3E53B4A602303FB90
:109680000020364B42685A60DBE5374A602303FB13
:109690000020324B82685A60D3E5334A602303FBD3
:1096A00000202E4B027B5A60CBE52F4A602303FB40
:1096B00000202A4BC2895A60C3E52B4A602303FB72
:1096C0000020264B02695A60BBE5274A602303FB52
:1096D0000020224B027D5A60B3E5234A602303FB3E
:1096E00000201E4B427D5A60ABE51F4A602303FBFE
:1096F00000201A4B026A5A60A3E51B4A602303FB51
:109700000020164B426A5A609BE5174A602303FB10
:109710000020124B826A5A6093E5134A602303FBD0
:1097200000200E4BC26A5A608BE50F4A602303FB90
:1097300000200A4B026B5A6083E50B4A602303FB4F
:109740000020064B82695A607BE5074A602303FBD1
:109750000020024BC2695A6073E500BF8897FF1F63
:109760009493FF1F7886FF1FC494FF1F7C2104F091
:10977000C3FF784B586064E5774A602303FB002001
:10978000744B426B5A605CE5734A602303FB002014
:10979000704B826B5A6054E56F4A602303FB0020D4
:1097A0006C4B827D5A604CE56C4B1844694B027ED1
:1097B0005A6046E5202104F09FFF664B586040E563
:1097C00060235843644B1A5C624B5A6039E566214A
:1097D00004F092FF5F4B586033E5652104F08CFF85
:1097E0005C4B58602DE503F01DF95A4B586028E595
:1097F000594A602303FB0020564BC26B5A6020E598
:10980000554A602303FB0020524B90F840205A60D9
:1098100017E5514A602303FB00204E4B90F841208E
:109820005A600EE54C4A602303FB0020494B426C12
:109830005A6006E50A2104F05FFF464B00F00F0076
:10984000C0F108005860FCE4454A642303FB002093
:10985000404B027A5A60F4E46423434340493F4A50
:1098600052F82020C85890473A4B5860E9E43C4AE7
:10987000642303FB0023394A52F82020586890479C
:10988000344B5860DDE4374B53F82020314B5A609D
:10989000D7E4354B53F820202E4B5A60D1E4304AA0
:1098A000642303FB00202B4B827D5A60C9E404F043
:1098B0008FFA284B5860C4E4294A642303FB002034
:1098C000244B828F5A60BCE4284B53F82020214B54
:1098D0005A60B6E4264B1A5C1E4B5A60B1E4502124
:1098E00004F00AFFA278234B53F82230C01A194B18
:1098F0005860A6E41A4A642303FB0020154BC26992
:109900005A609EE4164A642303FB0020114B026A4E
:109910005A6096E4124A642303FB00200D4B426A0E
:109920005A608EE40E4A642303FB0020094B828AAE
:109930005A6086E40A4B642202FB0030054B027E2B
:109940005A607EE4034B03221A707AE41A6822F00C
:10995000080284E48897FF1FC494FF1F7886FF1FC6
:109960009493FF1F2C93FF1FE495FF1F6493FF1F29
:109970009093FF1F5493FF1F38B5AA4A907802288E
:10998000144600F0EC80032800F0F080002840F03E
:10999000468153784D2B00F0A1803AD8452B79D0E1
:1099A00016D8412B6DD004D8402B63D003229E4B98
:1099B0005EE0422B69D0442BF8D19C49D2F80330A9
:1099C00041F81C3F04221C20BDE83840FFF7F9B9DC
:1099D000492B6CD014D8462B61D0472BE6D1934D40
:1099E000D2F803302946042241F8083F0820FFF747
:1099F000E8F92A8A29896879BDE8384003F010BF60
:109A00004B2B60D04C2BD1D1884BD1789970022050
:109A100033E0542B00F0838018D8512B6AD008D83B
:109A20004F2B60D0502BC1D1804BD1789975162027
:109A300023E0522B6BD0532BB8D17C4DD2F803309E
:109A40002946042241F8103F1020D0E7842B7CD017
:109A500008D8552B6ED0832BA8D1D2F80320744B95
:109A6000DA6138BD852B75D0FF2B9FD1D278714B31
:109A70001A7096E0D17845F2FF70BDE83840FFF7E4
:109A80008EB96A4BD1781970F7E7684BD178597065
:109A90000120F2E7654BD17859710520EDE7634964
:109AA000D2F8033041F80C3F04220C208CE7D27826
:109AB0005E4B1AB9DA75D97D1720DEE75A490122C3
:109AC000DA754A60F7E7594CD178E1700320FFF767
:109AD00066F9E078BDE83840FEF744BE534BD178D4
:109AE00059751520C9E7D2F80310504BC9B2597601
:109AF0001920C2E74D4D2A7DD20704D5E378DB0754
:109B000001D4FFF7B5F9E17829751420B5E7474985
:109B1000D2F8033041F8203F0422202054E7D2F845
:109B20000330012B7BD84149D37801F81A3F012239
:109B30001A2049E7D2F80330012B70D83B49D3787B
:109B400001F81B3F01221B203EE73B4BD2F80320CC
:109B50001A6038BDD2F80320354B1A6238BD5178EF
:109B6000364BD2F8032043F8212038BD5378272BF9
:109B700041D017D80B2B10D8092B12D2012B31D082
:109B800027D3022B7FF412AF2D4BD2F803209A601B
:109B9000FEF772FD264BD86238BD1B3B052B3FF606
:109BA00005AF38BD2B2B2BD008D8292BD2F803209A
:109BB000234BD2D07FF654AF5A6238BD2D2B29D01B
:109BC00023D32E2B7FF4F2AE1D4BD2F803205A6321
:109BD00038BD1B4BD2F803201A60FEF74DFD144B25
:109BE000586238BD164BD2F803205A60FEF744FD88
:109BF0000F4B986238BD124BD2F803209A6138BDE2
:109C00000F4BD2F803209A6238BD0D4BD2F80320D7
:109C1000DA6238BD0A4BD2F803201A6338BD042239
:109C2000C5E600BF6C96FF1F8897FF1F0C80FF1FC3
:109C30007886FF1F8297FF1F8497FF1F9497FF1F4F
:109C4000F095FF1F554B2DE9F74F00241C60544B36
:109C5000544D1C60544B554EDFF874B12C631C609E
:109C600085F8344005F1380705F10C0A05F144097F
:109C70005FFA84F82421404604F03EFD002304F8F6
:109C80000B30337E4AF82400494A002B54D1494B0B
:109C900049F8243045F8243042F824303B603B68D2
:109CA00001932821404604F027FD019B98473B681B
:109CB000B06229214046019304F01EFD019B9847A4
:109CC0003B68F0622A214046019304F015FD019B98
:109CD00098473B6830632B214046019304F00CFD0C
:109CE000019B984757F8043B70632C214046019331
:109CF00004F002FD019B98470134032CB06306F188
:109D00006406B5D12C4A00231946904642F8231028
:109D10000133B3F5807FF9D1284CA37E43BBE37EAA
:109D200053B3637DBBB3FEF73BFFA0B3012385F8BC
:109D30005C3003B0BDE8F08F214B49F82430214B53
:109D400045F82430204B42F82430204BA6E7B919BF
:109D500009EB0700042251440437FFF76BF80C2F7E
:109D6000F5D10C36FC2EDAD0002706F28C69EEE72E
:109D70000C26DFF860A0F7E74FF4FF6640F6D8073F
:109D8000A6F5FF613046042241440436FFF752F83D
:109D9000BE42F5D1C5E70023C9E700BF7497FF1F96
:109DA0009097FF1F7886FF1F7496FF1F9493FF1FE5
:109DB000C886FF1F5BEA00009497FF1F0C80FF1FFF
:109DC0004BEA000053EA00004FEA000057EA0000A7
:109DD0004F93FF1F7896FF1F014B93F85D0070476C
:109DE0007886FF1F70B5644E644B642505FB0065E3
:109DF0000446A96A99420CD8EA6A9A4209D82A6BA1
:109E00009A4206D86A6B9A4203D8AA6B9A4240F2E9
:109E10008380642505FB046502220021204604F0AE
:109E2000ABFCD5ED0A7AF8EE677A17EE900A06F0E9
:109E3000DBFF0022524B07F02BF84DA3D3E90023A0
:109E400007F050F907F036FA28210246204604F0C0
:109E50002DFCD5ED0B7AF8EE677A17EE900A06F036
:109E6000C3FF0022464B07F013F841A3D3E90023B8
:109E700007F038F907F01EFA29210246204604F0BF
:109E800015FCD5ED0C7AF8EE677A17EE900A06F01D
:109E9000ABFF00223A4B06F0FBFF35A3D3E90023CA
:109EA00007F020F907F006FA2A210246204604F0BE
:109EB000FDFBD5ED0D7AF8EE677A17EE900A06F005
:109EC00093FF00222E4B06F0E3FF29A3D3E90023E2
:109ED00007F008F907F0EEF92B210246204604F0BE
:109EE000E5FBA86B07EE900AF8EE677A17EE900A8A
:109EF00006F07AFF0022224B06F0CAFF1CA3D3E92A
:109F0000002307F0EFF807F0D5F902462C21204690
:109F1000BDE8704004F0CABB1A4E06EB840602226C
:109F2000002104F037FC336DA86A984728210246C7
:109F3000204604F0BBFB336DE86A984729210246AE
:109F4000204604F0B3FB336D286B98472A21024664
:109F5000204604F0ABFB336D686B98472B2102461B
:109F6000204604F0A3FB336DA86B9847CDE700BFF4
:109F7000000000A2941AED429493FF1FFFFF3F00E0
:109F8000000040427886FF1FF7B5044DAC786B782F
:109F9000022C05D9042200F031BD00BF6C96FF1FD2
:109FA000FF2B00F2B785DFE813F00602150234023A
:109FB00041024B0261026E029002B505B505B5057E
:109FC000B505A102B802C902D402DE02E602EE0221
:109FD000F80200030A03120327032B032F033303A2
:109FE00037033B034D03B505B505B5055A036803B3
:109FF000B505B505B505B505B505B505B505B50591
:10A00000B505B505B505B505B505B505B5057603C1
:10A01000B505B505B505B505B505B505B505B50570
:10A02000B505B505B505B505B505B505B505B50560
:10A03000B505B505B505B505B505B505B505B50550
:10A04000B505B505B505B505B505B505B505B50540
:10A05000B505B505B505B505B505B505B505B50530
:10A06000B505B505B505B505B505B505B505B50520
:10A07000B505B505B505B505B505B505B505B50510
:10A08000B50585038D039603A903BC03C503D5035A
:10A09000E703F003F9030A04190422042B04B505AD
:10A0A000B50534043D04460454045E046204B50559
:10A0B000B505B505B5057304B5057C0489049A0496
:10A0C000B505A404B505B505B505B505B505B505D2
:10A0D000B505B505B505B505B505B505B505B505B0
:10A0E000B505B505B505B505B505B505B505000159
:10A0F000090112011B012E0141014A0153015C01BA
:10A1000065016E0177018001B505B5058901B505C9
:10A110009201B505B5059B01B505B601BF01C801A2
:10A12000DE01F401B505B505B505B505B604BE04F7
:10A13000CA04B505B505B505B505D704E604F704A9
:10A14000B505FD01B505B505B505B5052C054F05EA
:10A15000B50572057B058305B505B505B505B505DE
:10A16000B505B505B505B505B505B505B505B5051F
:10A17000B505B505B505B505B505B505B505B5050F
:10A18000B505B505B505B505B505B505B505B505FF
:10A19000B505B505B505B505B505B505B505B505EF
:10A1A000B505B505B505B5058E05D5F803102046EE
:10A1B000C9B203B0BDE8F04003F048BFD5F80310C2
:10A1C0002046C9B203B0BDE8F04003F0ABBFD5F8FC
:10A1D00003102046C9B203B0BDE8F04003F0C6BF8B
:10A1E000204604F058F8D5F80310C9B228B9A87869
:10A1F00003B0BDE8F04003F0F7BFA87803B0BDE8B6
:10A20000F04003F0C5BF204604F045F8D5F8031030
:10A21000C9B228B9A87803B0BDE8F04003F004BF84
:10A22000A87803B0BDE8F04003F0CCBFD5F8031028
:10A230002046C9B203B0BDE8F04003F0DBBED5F85C
:10A2400003102046C9B203B0BDE8F04004F0ABB83B
:10A25000D5F803102046C9B203B0BDE8F04004F0C1
:10A260005DB8D5F803102046C9B203B0BDE8F04090
:10A2700004F066B8D5F803102046C9B203B0BDE8B3
:10A28000F04004F039B8D5F803102046C9B203B045
:10A29000BDE8F04004F066B8D5F803102046C9B216
:10A2A00003B0BDE8F04004F090B8D5F803102046A4
:10A2B000C9B203B0BDE8F04004F065B8D5F80310AA
:10A2C0002046C9B203B0BDE8F04003F0F5BED5F8B2
:10A2D00003102046C9B203B0BDE8F04003F086BFCA
:10A2E000D5F803000028FFF655AEBB4A642303FBF4
:10A2F0000424237E012B01D004F0ABFB0028D2BF45
:10A30000B64AB74A92FBF0F21421A87803B0BDE830
:10A31000F04003F0E5BDD5F803102046C9B203B004
:10A32000BDE8F04003F010BFD5F803102046C9B2D5
:10A3300003B0BDE8F04003F09BBED5F80300002851
:10A34000FFF628AEA44A642303FB0424237E012BDA
:10A3500001D004F07EFB0028CABFA14A9F4A92FBAD
:10A36000F0F21321D1E7D5F803102046C9B204F06A
:10A37000BBF80021A87803F0F9FDD5F803100246D8
:10A38000A87819B142F004020021BFE722F00402CC
:10A39000BCE7D5F803102046C9B203B0BDE8F040D1
:10A3A00004F0B2B8D5F803102046C9B203B0BDE836
:10A3B000F04004F051B860238A4A6343D35CD5F877
:10A3C000032013B937212046A2E0874B53F82430ED
:10A3D0001A44F7E760236343824AD35C1BB9D5F87C
:10A3E00003202121EFE72121204604F085F9D5F84B
:10A3F0000330C01A7C4B43F82400AC78502120462F
:10A4000004F07AF9D5F80330C01A784B43F82400E9
:10A410004CE0774B01221A55764B03EB84035B6CBF
:10A42000D5F80300984724210246CCE7714BD5F8B4
:10A43000030003EB84035B6C984722210246C2E7CA
:10A440006C4ED5F8030006EB8404636C9847002833
:10A45000B8BF4042E0602021A87804F04DF94307DE
:10A4600024D5AC7806EB8406736CD9E75A4A64238A
:10A4700003FB0423D5F803209A62204603B0BDE80D
:10A48000F040FFF7AFBC544B564AE878642101FB1B
:10A490000431602363434872D35C4BB98A7A897D67
:10A4A0008DE803000621204604F0D6F803B0F0BD85
:10A4B0001021204603F05AFDEB7820F4F852DB0817
:10A4C00042EA03221021204620E7434B4548EA7820
:10A4D000642101FB0431602363438A72C35C002B57
:10A4E000E4D1887D0190497A0091DBE70121204683
:10A4F00004F002F9D5F8033020F00A02DF0748BF64
:10A5000042F002029E0701D542F008020121A8781C
:10A5100003B0BDE8F04004F0C9B82046012104F0C2
:10A52000EBF8D5F8033020F00502DC0748BF42F015
:10A5300001029807EAD542F00402E7E7D5F80320C4
:10A54000012A3FF627AD2449642303FB0414E27576
:10A55000ACE7284BD5F8030003EB84035B6C98470A
:10A56000252102462FE71C4A642303FB0423D5F868
:10A5700003201A6381E7184A642303FB0423D5F8F8
:10A580000320DA6279E71B4BD5F8030003EB840361
:10A590005B6C98472721024615E70F4A642303FBAB
:10A5A0000423D5F803205A6367E7124BD5F803005C
:10A5B00003EB84035B6C98472621024603E7064AB7
:10A5C000642303FB0423D5F803209A6355E7D5F8E9
:10A5D00003202D21F7E600BF9493FF1FB500100064
:10A5E0000024F400C494FF1F4093FF1F5493FF1FE7
:10A5F0004F93FF1F7886FF1FD5F803202E21E2E638
:10A60000D5F803202F21DEE6D5F803203021DAE645
:10A61000D5F803203321D6E6D5F803203421D2E63D
:10A620000121204604F068F8D5F8033020F0C0027C
:10A63000D90748BF42F040029B077FF567AF42F061
:10A64000800263E70121204604F056F8D5F8033074
:10A650001B0220F4407203F440731A4356E70121B1
:10A66000204604F049F8D5F8033020F01002002B02
:10A670003FF44CAF42F0100248E70121204604F0BD
:10A680003BF8D5F8033020F02002002B3FF43EAF1A
:10A6900042F020023AE760236343BB4AD35C002BBD
:10A6A0003FF404AFD5F80310204603B0BDE8F040F6
:10A6B00002F008BAB44BD5F80320602101FB043343
:10A6C0005A6080E6B049D5F80320602303FB0413E9
:10A6D00061219A6077E6AC4A602303FB0423D5F836
:10A6E00003201A731C21204604F006F8D5F8032035
:10A6F000C0F3080040EA02421C2108E7A24A602396
:10A7000003FB0423D5F80320DA811C21204603F043
:10A71000F3FFD5F8033000F47F02C3F308031A43B4
:10A72000EAE79949D5F80320602303FB0413592174
:10A730001A6148E660239448D5F803206343C118A2
:10A74000C35CD2B20A75002B3FF4B0AE8B7D019290
:10A750004A7D0EE060238C48D5F803206343C1187E
:10A76000C35CD2B24A75002B3FF4A0AE8B7D097D4D
:10A7700001910092002295E68349D5F803206023D9
:10A7800003FB04135A211A621DE67F49D5F8032002
:10A79000602303FB04135B215A6214E67A49D5F85F
:10A7A0000320602303FB0413D1B29A62C2F3072291
:10A7B00093F82C300191009200225D2173E67249DA
:10A7C000D5F80330602202FB0412D362926AD1B240
:10A7D000C2F3072201910092DBB2EDE76A49D5F896
:10A7E0000320602303FB04135E211A63EBE5664933
:10A7F000D5F80320602303FB041318219A61E2E5D6
:10A800006149D5F80320602303FB04131921DA61A1
:10A81000D9E55D49D5F80320602303FB04135C21CF
:10A820005A63D0E55849D5F80320602303FB04138D
:10A830005F219A63C7E560225348D5F8033062432D
:10A840008118825CDBB28B75002A3FF42FAE0A7D43
:10A850007DE7D5F80330022B3FF69CAB4B4B1C44F5
:10A86000EB78237622E6D5F803202021ABE5D5F856
:10A8700003204549012A08BF45484FF0600313BF34
:10A880005C4302555C4300230CBF0A550B550DE693
:10A890003D49D5F80320602303FB04135221DA63FA
:10A8A00091E5394AE978602303FB04235A6C83F865
:10A8B0004010019193F8413000930BE0324AE9785F
:10A8C000602303FB042383F841105A6C93F8403053
:10A8D0008DE80A00D3B26321C2F30722E3E52A49D7
:10A8E000D5F80320602303FB04135A6493F8401047
:10A8F000DFE7D5F80330082B3FF64CAB0A212046A2
:10A9000003F0FAFED5F8033020F00F02C3F108037C
:10A910001A430A21FBE51F4A642303FB0424D5F8EC
:10A9200003302372C2E5194BD5F8030003EB84030F
:10A930005B6C984764235C43164B1851B6E5134B88
:10A94000D5F8030003EB84035B6C9847114A64233A
:10A9500003FB04246060A9E50E4B0B4AE8786421F0
:10A9600001FB0431602363438875D35C002B7FF4C3
:10A970009DAD8A7AB6E5D5F80310204603B0BDE850
:10A98000F04003F0DDB900BFC494FF1F7886FF1FBD
:10A990004F93FF1F9493FF1F5F4FD5F8032064264A
:10A9A00006FB04718B8F9A423FF480AD60236343B2
:10A9B0005A48C35C0BBB0C238A872046009392B293
:10A9C00004230A2103F0F4FEA87806FB0073542147
:10A9D000DA69002AB8BF524203F068FEA87806FB85
:10A9E0000076F369002B4FF000524FF0070149DA6F
:10A9F00003B0BDE8F04003F0BFBE0622484B1A701A
:10AA000054E560236343454A464ED75C97B15021D5
:10AA1000204603F071FED5F80330C01A46F8240032
:10AA2000AC782121204603F067FED5F80330C01A28
:10AA30003D4BEBE4D5F803205021204603F036FED1
:10AA4000AB7846F8237031E5334FD5F80320642600
:10AA500006FB0473DB699A423FF428AD602363432D
:10AA60002E49CB5C002BC8D1002A2046B8BF5242E9
:10AA7000542103F01BFEA878D5F8033006FB0076BE
:10AA8000F361AFE703B0BDE8F04003F083BE2249B5
:10AA9000D5F80320642303FB041353211A6292E4C4
:10AAA0001D4A642303FB0424D5F803306362FDE4EC
:10AAB0001949D5F80320642303FB041315219A8256
:10AAC0001A4B5A437FE4D5F80330A3B1012B7FF42E
:10AAD00061AA1149642202FB041215491376154A32
:10AAE00002EB84035964144942F82410134A1A658E
:10AAF000134A9A63DAE40849642202FB04120D49FE
:10AB0000137601EB84020F4B536441F82430136534
:10AB10009363CBE4032271E79493FF1FC494FF1F58
:10AB20008897FF1F5493FF1F4093FF1F007102007F
:10AB30004BEA00007886FF1F53EA00004FEA00004E
:10AB400057EA00005BEA00002DE9F743C74EDFF843
:10AB500050833278D6F8033088F801206427212A00
:10AB600088F80070C8F804303446454601F0578034
:10AB700000F2C4800E2A00F014853AD8072A00F0AB
:10AB8000A48314D8032A00F01C8208D8012A00F0FC
:10AB90009C81022A00F0D98102232B70CDE1052A85
:10ABA00000F0908340F22982FEF734FAC5E10A2AC8
:10ABB00000F0918307D8082A00F08A83092AEBD194
:10ABC000FEF7DAFEB9E10C2A00F0BC8440F2A4845E
:10ABD000B078022800F2B6817378012B00F0C884A7
:10ABE000C0F0C384022B00F0C684032388F8003031
:10ABF000A3E1182A00F02F862BD8142A00F08485B0
:10AC000015D80F2A00F0E984132AC5D17178984A23
:10AC1000092900F24085DFE811F03B0546054905AA
:10AC20004C05500557055A055D0560055505162A62
:10AC300000F00D8640F288858E4A116E072900F2D9
:10AC40007C81481C02EB81011066106B486613631F
:10AC500073E11C2A00F0018722D81A2A00F0198615
:10AC600040F20686834D95F8342072B95E1C04BF0D
:10AC70007F4B1B680A205843C5F88800FDF7FCFC91
:10AC80000123C5F88C0085F834306378042B00F27A
:10AC90005481DFE813F00F0650067E06B406250641
:10ACA0001F2A00F00F8700F260871E2A7FF474AF1E
:10ACB0007278142A00F23F84B078022800F2D3861A
:10ACC00002EB42046C4D044445F824306B4B9B7EF0
:10ACD000002B00F03281002A00F02F81032111FBAC
:10ACE00002010C23013A5A4302F5D363042205EB17
:10ACF000810102FB0030FEF764F81EE1802A01F0BA
:10AD0000788044D8402A01F05C8029D8242A00F0B9
:10AD1000F2870CD8222A00F0E687232A7FF43CAF82
:10AD2000534B1B68C6F80330FEF726FE05E1262AC2
:10AD300001F01F80C1F01280272A7FF42DAFB27876
:10AD4000022A00F2FF807378142B00F2F48303EBE5
:10AD500043031344464A1168474A42F82310ECE083
:10AD6000442A01F03A8007D8422A01F0328041F2A9
:10AD70002C8001F052FEE0E0462A01F03680C1F05E
:10AD80003080472A7FF408AF01F04BFED5E0872AD8
:10AD900001F0CF8046D8832A01F04A800AD8812A60
:10ADA00001F02D80822A7FF4F7AE324B022283F825
:10ADB0005C20C2E0852A01F06F80304A41F2588061
:10ADC0002F49304C01250D70B3F5C05F917821708B
:10ADD00081F06880127D12EA050641F06380184612
:10ADE0006946FEF73EF89DF8003063709DF801302B
:10ADF000A3709DF80230E3709DF8063023719DF832
:10AE0000053063719DF80430A3719DF80330E37140
:10AE100026722B46E15C227A01330A44082B227207
:10AE2000F8D18AE08C2A01F0EA803BD8892A01F027
:10AE3000CB80C1F041808A2A7FF4AEAE7278124B8B
:10AE4000002A41F0D9801A70104AE3781370094A39
:10AE500092F874110E4A11700E4900220A700E49C0
:10AE60000A700E4A11780B43137066E06C96FF1F50
:10AE70007497FF1F7886FF1F7896FF1F0C80FF1FB7
:10AE80007897FF1F7997FF1F3893FF1F6093FF1F6D
:10AE90003896FF1F5293FF1F6896FF1F3993FF1FBD
:10AEA0008897FF1FF22A01F02081FF2A01F06281BA
:10AEB0008D2A7FF471AE7278032A01F21181DFE8E6
:10AEC00012F0E208C908FC080A09B078022839D84B
:10AED00001F026FE0125B078AB4B4FF00062294609
:10AEE0001D5403F049FCB078A84A642303FB0023F7
:10AEF000DB7D2BBB2A46202103F0D8FBA578A44B91
:10AF0000D4F8030003EB85035B6C984724210246C9
:10AF1000284603F0CBFB4FF080520721A07803F0C6
:10AF20002BFC4FF000620721A07803F033FC4FF0B8
:10AF300000620121A07803F02DFC03B0BDE8F0838E
:10AF40000222D8E704232B70F7E7B0780228F9D85B
:10AF500001F0E6FD0125B0788B4B4FF000622946E9
:10AF60001D5403F009FCB078884A642303FB0023D6
:10AF7000DB7D23BB2A46202103F098FBA578844B78
:10AF8000D4F8030003EB850340425B6C984724210F
:10AF90000246284603F08AFBA0784FF08052072132
:10AFA00003F0EAFBA0784FF00062072103F0F2FB08
:10AFB0004FF000620121A07803F0ECFBBDE7022214
:10AFC000D9E7B0780228BDD802F068FBB0786E4BA4
:10AFD00001221A546D4B07FB0037FB7D5BB9202122
:10AFE00003F064FBA0780022242103F05FFBA0782B
:10AFF00001F096FDA1E70222F1E7B078022802D91C
:10B000007278022A99D16678012E00F09C8054D380
:10B01000022E92D1142B95DC020640F10981DFF853
:10B020006C81594FDFF874910025A3782B41DB0721
:10B030003FD5EEB2304601F073FD642303FB058378
:10B04000DB7D002B40F0E68005222021304603F016
:10B050002DFBEB5D43B14F4B242153F825203046A7
:10B0600003F024FB0023EB554FF0805207213046BC
:10B0700003F090FB4FF000620721304603F07CFBA9
:10B0800060236B43444A13F80930002B40F0C4801E
:10B09000D4F8033003EB43032B4452F82320372129
:10B0A000304603F003FB4FF000620121304603F00D
:10B0B00071FB0135032DB8D13FE701F031FD4FF0B1
:10B0C0000062A078012103F057FBA0782F4A642387
:10B0D00003FB0023DB7D7BBB0522202103F0E6FA86
:10B0E000294DA0782B5C4BB1294B03EB8003242125
:10B0F000DA6803F0DBFAA3780022EA544FF08052BA
:10B100000721A07803F046FB4FF00062A0780721EA
:10B1100003F032FBA078214A60234343D35CD4F888
:10B1200003205BB9372103F0C1FA4FF0006201211F
:10B13000A07803F02FFB00E70622CEE7184B53F868
:10B1400020301A44EEE701F0EBFC4FF00062A078EB
:10B15000314603F011FBA0780C4A642303FB002363
:10B16000DB7D73B90522202103F0A0FA084EA078F8
:10B1700033181B7E012B40D014D3022B3FD0002567
:10B1800016E00622EFE700BF4F93FF1F9493FF1FC7
:10B190007886FF1F8486FF1F7896FF1FC494FF1FC9
:10B1A0004093FF1F372103F0A7FAD4F8035005445A
:10B1B000A078A64F3B5C43B106EB80062421F268E1
:10B1C00003F074FAA3780022FA54A0784FF080526A
:10B1D000072103F0DFFAA0784FF00062072103F0A7
:10B1E000CBFA2A46A078372103F060FA4FF00062CC
:10B1F0000121A07803F0CEFA9FE62121D3E7502168
:10B2000003F07AFAA278924B53F82250451BD4F8F7
:10B210000300CCE7062218E7D4F8033003EB43031E
:10B220002B4452F823208B4B53F825301A4436E731
:10B2300002283FF687AE01F073FCA078864A6423AB
:10B2400003FB0023DB7D002B35D10522202103F0F9
:10B250002DFA7E4DA0782B5C4BB1804B03EB800325
:10B260002421DA6803F022FAA3780022EA544FF08E
:10B2700080520721A07803F08DFA4FF00062072179
:10B28000A07803F079FAA078754A60234343D15C33
:10B29000D4F80330734A03EB4303034452F82320EA
:10B2A00059B9372103F002FA4FF000620121A0786A
:10B2B00003F070FA41E60622C8E7664B53F82030E7
:10B2C0001A44EEE7FEF760FE37E6FDF795FE34E63A
:10B2D000FDF792FE31E6B378022B00F0D380032B0A
:10B2E00000F0D580002B40F010817378502B00F0D7
:10B2F000828028D8462B6FD010D8422B66D006D833
:10B30000402B48D0412B5DD003232B7049E0442BC8
:10B310005FD0452BF8D1544B5B7955E04B2B61D076
:10B3200009D8472B5BD0492BEED14F4BDB7D003347
:10B3300018BF012348E04D2B5AD056D34F2BE3D1F1
:10B34000494B5B7E40E0802B64D012D8532B58D001
:10B3500006D8512B52D0522BD6D1434B1B6A33E027
:10B36000552B54D050D3562BCED13F4B93F824308D
:10B370002AE0832B59D006D8812B4FD0822BC3D102
:10B38000364B1B6B20E0852B54D050D3FF2BBBD109
:10B39000364B1B78CBE745F2FF70FDF739FDC8F857
:10B3A0000400334B1B78002B3FF4C7AD314B6A6868
:10B3B0001A60314B002A40F0AA801A6842F0080255
:10B3C0001A60BAE5284B1B786B60EAE7264B5B787E
:10B3D000FAE7254BDB69F7E7234BDB68F4E7224B01
:10B3E0009B68F1E7204BDB78EEE71F4B9B78EBE7A0
:10B3F0001D4B5B7DE8E71C4B9B7DE5E71A4B1B7DF6
:10B40000E2E7194B1B69DFE7174B9B7EDCE7164B26
:10B41000DB7ED9E7114B93F85C30D5E70F4B93F8FF
:10B420005C301E1F73427341CEE70C4BD2E7134BC7
:10B430001B68C9E7094A1248136A43F2390100FB45
:10B440000313136223F00043BEE700BF4F93FF1FB7
:10B450005493FF1F4093FF1F9493FF1F7886FF1F95
:10B46000C494FF1F7896FF1F0C80FF1F8297FF1F59
:10B470008397FF1F7497FF1F7496FF1F8497FF1F0A
:10B480006D4EC6417278994B53F822309CE7737821
:10B49000282B2ED015D8022B29D006D82BB3012B60
:10B4A0007FF432AF924B5B688EE7092BFFF42CAF31
:10B4B0000B2B7FF676AF272B7FF426AF8C4B9B6947
:10B4C00082E72B2B19D007D8292B14D02A2B7FF4F5
:10B4D0001BAF874B5B6A77E72D2B14D010D32E2B35
:10B4E0007FF412AF824B5B6B6EE7814BA0E7804B22
:10B4F00076E77F4B6EE77E4B30E77D4B9B6A63E7D9
:10B500007B4BDB6A60E77A4B3BE70423FDE61A6876
:10B5100022F008021A6010E5B378022B0ED1707881
:10B52000372808D800F5FF707249800004220144D2
:10B53000FDF747FC01E503232B70FEE4042388F8A4
:10B540000030FAE4B378022B0BD170783728F2D8A8
:10B5500000F5FF706749800004220144FDF76AFC92
:10B56000EBE4042388F80030E7E402F08FF8E4E429
:10B5700002F094F8E1E402F099F85F4BC8F8040097
:10B580001B78002B3FF4D9AC5C4B18605C4B1A68FD
:10B5900018B942F008021A60CFE422F008021A60DB
:10B5A000CBE4B278022A14D17078072806D813B9F0
:10B5B000FDF72AFAC1E4FDF713FABEE4FF287FF491
:10B5C000BCAC5D1C0ABF4D4BD8B21878FDF730FA01
:10B5D000B3E4042388F80030AFE4B378012B2BD018
:10B5E0002BB1022B4BD0042388F8003010E0707888
:10B5F000082803D8FDF72DFA686009E00A2816D15B
:10B60000404B1B6983F40073C3F34023C8F8043034
:10B61000394B1B78002B3FF490AC384B6A681A60AA
:10B62000374B82BB1A6842F008021A6085E4FF2893
:10B63000EED1FDF745FADFE77078092802D002F075
:10B64000BFF8D9E70020FDF753FA04460120FDF7C3
:10B650004FFA06460220FDF74BFA8642D4BF00237C
:10B6600001239C4209DD331C18BF01231BB986420C
:10B670003446B8BF04466C60CAE7031CF4E7707830
:10B68000FDF700FAB8E71A6822F008021A6054E4DD
:10B690001068184410601268194B0ABB1A6842F00F
:10B6A00008021A6049E41068C01AF3E710685843AA
:10B6B000F0E7106890FBF3F0ECE7116891FBF3F012
:10B6C00003FB10131360E6E710681840E2E7106808
:10B6D0001843DFE710685840DCE71368DB43F1E705
:10B6E0001A6822F008021A6027E400BF9497FF1F2F
:10B6F000F095FF1F9C8FFF1F8397FF1F7497FF1FFD
:10B700007496FF1F80F00F40AA4A1168AA4A8B4224
:10B7100013680ADA23F0030343F004031360136889
:10B7200069B943F00803136007E40BBF23F0060375
:10B7300023F0050343F0010343F00203EEE723F097
:10B7400008031360FFF7F9BB72780C2A3FF6F5ABDC
:10B75000DFE802F0071019222B343E475059626B84
:10B760007400954A126814077FF5E7AB934A136398
:10B77000FFF7E3BB904A126810073FF5DEAB8F4A34
:10B780001363FFF7DABB8C4A1268D1077FF5D5AB9C
:10B790008A4A1363FFF7D1BB874A1268D2073FF585
:10B7A000CCAB864A1363FFF7C8BB834A12685707BE
:10B7B0007FF5C3AB814A1363FFF7BFBB7E4A1268B4
:10B7C00012F0050F3FF4B9AB7C4A1363FFF7B5BB2A
:10B7D000794A126896077FF5B0AB784A1363FFF792
:10B7E000ACBB754A126895073FF4A7AB734A136365
:10B7F000FFF7A3BB704A1268D4067FF59EAB6F4A71
:10B800001363FFF79ABB6C4A126890067FF595ABFD
:10B810006A4A1363FFF791BB674A126851067FF5C6
:10B820008CAB664A1363FFF788BB634A1268120643
:10B830007FF583AB614A1363FFF77FBB5E4A1268F3
:10B84000D7057FF57AAB5D4A1363FFF776BB5B4A9A
:10B850001363FFF772BB594A136E002B3FF46DABB5
:10B86000013B136602EB83035B6E1363FFF765BB5B
:10B8700073782E2B04D8524A0121D154FFF75DBBB7
:10B88000FF2B7FF458AE4D4B012283F88420FFF745
:10B8900054BB73782E2B04D8494A0021D154FFF7AA
:10B8A0004CBBFF2B7FF447AE444B002283F884202F
:10B8B000FFF743BBFCF7E0FED5F88C30C01A002838
:10B8C000D5F88830B8BF4042984295BF2B6B002313
:10B8D00003F1FF3385F8343098BF2B63FFF72DBB9E
:10B8E000A07801F0E3FE40B9334A85F834001368CC
:10B8F00023F010031360FFF720BBD5F88830ABB1FD
:10B90000FCF7BAFED5F88C30C01A0028D5F888307C
:10B91000B8BF4042984209D9274A002385F83430FD
:10B92000136843F010031360FFF707BB2B6B013B59
:10B930002B63FFF702BBA0780F2102F0DDFE10F0B1
:10B94000010409D01C4A002385F83430136823F021
:10B9500010031360FFF7F1BAD5F88830A3B1FCF7F4
:10B960008BFED5F88C30C01A0028D5F88830B8BFC7
:10B970004042984208D9104A85F83440136843F091
:10B9800010031360FFF7D9BA2B6B013B2B63FFF752
:10B99000D4BAA0780F2102F0AFFE10F0800411D0CD
:10B9A000054A002385F83430136823F01003136030
:10B9B000FFF7C3BA7497FF1F7496FF1F7886FF1FA7
:10B9C0003996FF1FD5F88830A3B1FCF755FED5F89E
:10B9D0008C30C01A0028D5F88830B8BF4042984251
:10B9E00008D9B24A85F83440136843F01003136055
:10B9F000FFF7A3BA2B6B013B2B63FFF79EBAA0782E
:10BA00000F2102F079FE10F4807409D0A74A0023B8
:10BA100085F83430136823F010031360FFF78DBAF4
:10BA2000D5F88830A3B1FCF727FED5F88C30C01AC2
:10BA30000028D5F88830B8BF4042984208D99B4AC0
:10BA400085F83440136843F010031360FFF775BAAC
:10BA50002B6B013B2B63FFF770BA954B002283F8E9
:10BA60005C20FFF76ABAFF287FF46CAA914E3AB3C4
:10BA700000254FF003080C27607818FB00510138AF
:10BA8000784300F5D36000EB8500042206EB8101CA
:10BA90000135FDF796F9032DEED1FFF74EBA611986
:10BAA0007819042231440435FDF78BF90C2DF6D1B9
:10BAB0000C34FC2C3FF441AA002504F28C67EEE71D
:10BAC0000C24F9E77378142B3FF635ADB278022ACF
:10BAD0001CD803EB43031344764A52F82320764BD9
:10BAE000C8F804201B78002B3FF427AA734B1A6078
:10BAF0006E4B2AB91A6842F008021A60FFF71DBAA5
:10BB00001A6822F008021A60FFF717BAFF2A7FF4BA
:10BB100019AA684E3BB300254FF003080C27607844
:10BB200018FB00510138784300F5D36000EB850025
:10BB3000042206EB81010135FDF77CF9032DEED1DE
:10BB4000FFF7FBB961197819042231440435FDF778
:10BB500071F90C2DF6D10C34FC2C3FF4EEA9002524
:10BB600004F28C67EEE70C24F9E77678142E3FF6A2
:10BB7000E2ACA77838062AD54E4FDFF8448100257D
:10BB8000A3782B41D90709D566782121E8B202F0C4
:10BB9000B3FD06EB46062E4447F8260098F81A3007
:10BBA00083B1637873B1032111FB03510C20013B76
:10BBB000584300F5D360042207EB810100EB8500B8
:10BBC000FDF7FFF80135032DDAD1FFF7B6B9022FE3
:10BBD0003FF6B8A92121384602F08EFD384B354D8D
:10BBE0009B7E06EB46063E4445F82600002B3FF4BC
:10BBF000A4A96278002A3FF4A0A9A078032111FB30
:10BC000002010C23013A534303F5D363042205EBED
:10BC1000810102FB0030FDF7D4F8FFF78EB972788E
:10BC2000264B0A2A0CD8DFE802F006151A1F252D2C
:10BC300032373C4F530023491A6809680A441A6096
:10BC40001A681A4B002A48D11A6842F008021A6092
:10BC5000FFF773B91B491A680968521AEFE7194AC6
:10BC6000196812684A43EAE716491A68096892FB9C
:10BC7000F1F2E4E7134A1868116890FBF1F201FB56
:10BC80001202DCE70F491A6809680A40D7E70D4934
:10BC90001A6809680A43D2E70A491A6809684A40DB
:10BCA000CDE708490A68D2430A60C9E77496FF1FC6
:10BCB0007886FF1F7896FF1F8397FF1F7497FF1FDB
:10BCC0000C80FF1F9097FF1F1968B54A1160B7E7F6
:10BCD000B34A196810681860F8E71A6822F0080279
:10BCE0001A60FFF72AB9AF4B1B68C6F80330FEF79E
:10BCF0004BF9FFF722B97378052B3FF61EA9DFE851
:10BD000003F0030A11181F26A74A136803F00F0354
:10BD10001360FFF712B9A44A136823F010031360ED
:10BD2000FFF70BB9A04A136823F020031360FFF755
:10BD300004B99D4A136823F040031360FFF7FDB870
:10BD4000994A136823F080031360FFF7F6B8964A08
:10BD5000136823F480731360FFF7EFB871782E290E
:10BD60003FF6E9AB914A02EB8102C2F89030FFF74F
:10BD7000E4B88E4B8B4AD3F84C111160884AD3F843
:10BD800050111160D3F854211A63874AD3F858111F
:10BD90001160D3F85C2183F83420D3F86021C3F814
:10BDA0008C20D3F86421C3F8882093F86811804A66
:10BDB000505C08B101205054002283F86C21FFF739
:10BDC000BCB800F01BFEFFF7B8B800F018FEFFF794
:10BDD000B4B800F021FEFFF7B0B800F01FFEFFF787
:10BDE000ACB800F01CFEFFF7A8B800F019FEFFF792
:10BDF000A4B86E4B002283F85C20FFF79EB87278DF
:10BE000032B1012A0AD0032388F80030FFF795B831
:10BE1000664B012283F85C20FFF78FB8B3F5C05F53
:10BE2000BFF490A8614981F85C200B63FFF785B8E7
:10BE30005E4A5F48002382F8843082F86C3102F158
:10BE400090044FF0FF35194644F82350C154013394
:10BE50002F2BF9D1534B82F85C101960504B1163B2
:10BE60001960514B116682F834101960FFF765B8FC
:10BE7000127D92070BD4B3F5C05FBFF463A84B4AA1
:10BE8000042182F85C10C2F87031FFF756B808231D
:10BE900088F80030FFF751B8444B002283F85C204B
:10BEA000FFF74BB82B460022E2540133082BFBD19D
:10BEB00023782372FFF741B87378012B1AD006D389
:10BEC000022B24D0032388F80030FFF736B8394B13
:10BED00001221A70384B394A9B781370384B196815
:10BEE00000230139013311F8010FD054082BF9D187
:10BEF000FFF723B80C2288F8072088F80530F022D5
:10BF0000072388F8062088F80430FFF716B8294B75
:10BF10002C4801221A70284B284A9B781370002362
:10BF200001331918082B11F8091CD154F8D1FFF767
:10BF300004B87378032B3FF600A8DFE803F002147F
:10BF4000252B1A4B93F85C2088F8072093F83420AF
:10BF5000D3F8703188F806201A0A88F8052088F886
:10BF60000430FEF7EABF114B93F85C2088F80720F5
:10BF700093F834201B6B88F806201A0A88F80520ED
:10BF800088F80430FEF7D9BF064B1B68C8F80430A8
:10BF9000FEF7D3BF024B1B68C8F80430FEF7CDBFD5
:10BFA0009097FF1F7497FF1F7496FF1F7886FF1FDF
:10BFB0003996FF1F7897FF1F0C80FF1F7997FF1F8F
:10BFC0000880FF1F008000007278002A7EF4B5AF61
:10BFD000B17800297EF4B1AF40F2D24293427EF4B0
:10BFE000ACAF45F2FF70FCF7DAFEFCF741FF012031
:10BFF000FCF71EFCFEF7A1BF0122FEF724BF7478F8
:10C0000034B1012C16D0032388F80030FEF795BF19
:10C010000422694645F2FB70FCF70CFF009BD6F842
:10C0200003209A4206BF0123C8F80430C8F8044030
:10C03000FEF783BFB3782A2B07D10422534945F278
:10C04000FB70FCF7BEFEFEF778BF032388F80030D4
:10C05000FEF773BF4E4CD4F87801002104F5BE7290
:10C0600081423EF46AAF52F821509D4201F1010530
:10C0700021D102EB8503043B0138814215D3C4F87A
:10C080007801FEF75ABF424AD2F8781109299DBFBC
:10C09000481CC2F8780102EB8102092394BFC2F860
:10C0A0007C3188F80030FEF748BF53F8042F43F87E
:10C0B000042C0131E1E72946D2E7354A0023C2F8D2
:10C0C0007831194602F5BE7242F8231001330A2B6B
:10C0D000FAD1FEF732BF0A23C8F80430FEF72DBFAD
:10C0E000032388F80030FEF728BF7378812B7EF495
:10C0F00029AFB378922B7EF425AFB379A32B7EF4CE
:10C1000021AF7379B42B7EF41DAF3379C52B7EF448
:10C1100019AFF378D62B7EF415AFFCF77CFDFCF756
:10C12000ABFA0446FCF7A8FA001B0028B8BF40424F
:10C13000B0F57A7FF6DBFCF779FB164B00221A602C
:10C140004FF0FF32C3F87021C3F87022C3F8742196
:10C15000C3F87422C3F87821C3F87822C3F87C218D
:10C16000C3F87C220C4B0D4A1A600120FCF760FBDF
:10C17000FEF7E3BE40F2D24293427EF4DEAE044BC1
:10C18000012283F8A421FEF7D8BE00BF6F96FF1FDF
:10C190007886FF1F10E000E00080FF1F7856341201
:10C1A000F7B50F4C07460E4694E803008DE80300F0
:10C1B0000C49C1F803300C4B8A7000220F704E708E
:10C1C0001A70FEF7C1FC094A217882F85D109DE8DB
:10C1D0000300636884E80300184603B0F0BD00BFA5
:10C1E0008897FF1F6C96FF1F8397FF1F7886FF1F9E
:10C1F000F7B504461F4A63781370A3785370E37849
:10C2000093702379937163795371A3791A4D1371E4
:10C21000E379D3700E4695E80300184B00221A709C
:10C220008DE80300FEF790FC154B1A786F462B46FD
:10C230009AB9327072702A78B2706A78F270EA79BC
:10C240003271AA7972716A79B2712A79F27197E8BA
:10C25000030083E8030003B0F0BD012AF7D10948C9
:10C26000721EF11D10F8014F02F8014F8A42F9D1F8
:10C27000EDE700BF6C96FF1F8897FF1F8397FF1F96
:10C280007897FF1F7997FF1F2DE9F043994B9A4C40
:10C290001B788FB06BB1994B1B78063BDBB2192B27
:10C2A00004D8974A22FA03F3D90702D4002384F86A
:10C2B000743194F87431934E5A1E012A51D8924920
:10C2C000012BCA68079214BF082307238DF8183082
:10C2D000327894F8A5318DF8193000238DF81A3092
:10C2E000002A33D18B688DF82030884B8DF82720B9
:10C2F00019788DF8211059788DF82210D9798DF898
:10C30000231099798DF8241059791B798DF825100F
:10C310008DF8263006A801F071FB002800F01F837D
:10C320007B4B1A789846002A00F01E81794B7A4F91
:10C330001B78013B062B00F21381DFE813F0F100BC
:10C34000F10058011101110111017F01012AE1D110
:10C350007248013306AA1A44195CD171082BF8D12E
:10C36000D8E7032B3DD1337883BBDFF89C81674F3F
:10C3700098F8020098F801503B7805441D447B78FA
:10C380001D44FB791D44BB791D447B791D443B79D9
:10C390001D44FCF7ABF998F80100FCF7A7F93878D1
:10C3A000FCF7A4F97878FCF7A1F9F879FCF79EF985
:10C3B000B879FCF79BF97879FCF798F93879EDB200
:10C3C000FCF794F92846FCF791F9A9E7012BA7D1CE
:10C3D000524F0025785D0135FCF788F9092DF9D118
:10C3E0009EE7042B2BD1484FDFF82081B8787D7869
:10C3F000002301220544154488F8013088F8002004
:10C40000C8F80430FCF772F97878FCF76FF998F8FF
:10C410000000FCF76BF998F80100FCF767F998F851
:10C420000700FCF763F998F80600FCF75FF998F845
:10C430000500FCF75BF9EDB298F80400C0E7072BA4
:10C4400037D1337853BB304B9F7893F801802F4B13
:10C450008DF800701D785878D9798DF802504744CE
:10C460003D449A798DF80300284493F805C08DF86F
:10C470000410014493F804E08DF805200A440CEB05
:10C48000020373448DF801808DF806C08DF807E033
:10C490008DF808306846FCF7BBFB41E7012BF9D16A
:10C4A0001E4900235A5C0DF803200133092BF9D1F2
:10C4B000F0E7082B7FF434AF144A1349002301201E
:10C4C0005370107053608A7849788DF800200A44C0
:10C4D00002448DF801108DF802008DF803308DF8BC
:10C4E00004308DF805308DF806308DF807308DF862
:10C4F0000820CFE78297FF1F7886FF1F6C96FF1FEB
:10C50000110200027897FF1F0C80FF1F8897FF1F02
:10C510006896FF1F3896FF1F5293FF1F7997FF1FE2
:10C52000AE4A397893688DF8303080238DF83130F9
:10C530008A238DF8323000238DF833308DF8343073
:10C540008DF835308DF836108DF8293007218DF8AB
:10C550002A300AA8D3688DF828100B9301F04EFA00
:10C5600000233B7088F80030002384F87431337066
:10C5700094F8A43113B10120FCF75AF906A801F090
:10C58000C9F90646002800F04181954B9DF820200E
:10C590001A709DF821205A709DF822209A709DF8FB
:10C5A00023209A719DF824205A719DF825201A7134
:10C5B0009DF82620DA709DF8193084F8A531FCF733
:10C5C0005BF8884B1860884B00221A709DF8183071
:10C5D000072B0CBF0123022384F8743194F85C30DC
:10C5E0005A1E012A4AD9052B48D0012247E0DFF81C
:10C5F000EC913B7899F8020099F8015005440A350E
:10C600001D44FCF773F899F80100FCF76FF88020DF
:10C61000FCF76CF88A20FCF769F80020FCF766F854
:10C620000020FCF763F80020FCF760F8EDB23878E2
:10C63000FCF75CF82846FCF759F891E7674A507810
:10C6400093788DF80C303A788DF80D0080210344F2
:10C650008DF80E100A338A218DF80F101344002133
:10C6600003A88DF810108DF811108DF812108DF8A8
:10C6700013208DF81430FCF7CBFA71E700225B4BE6
:10C680001A7094F85C30042B04D1554B19780A06C3
:10C6900040F1688194F87421082A04D840F25113BB
:10C6A000D340DF0701D4FEF74FFA94F87431092B19
:10C6B0006FD1FBF7E1FF636A4D4DC01A00282A686D
:10C6C000B8BF4042904208D94A4B1A78012A04BFA9
:10C6D00002221A70FBF7D0FF6062FBF7CDFFA36A5E
:10C6E0006A68C01A0028B8BF4042904208D9414B3E
:10C6F0005A78012A04BF02225A70FBF7BDFFA062DC
:10C70000FBF7BAFFE36AAA68C01A0028B8BF404224
:10C71000904208D9374B9A78012A04BF02229A70B6
:10C72000FBF7AAFFE06294F8843093B394F86C317D
:10C730007BBB304A30481D46D15C022940F006815F
:10C7400050F823104E1C00F000812C4A84F8683108
:10C750001268C4F84C212A4A1268C4F85021226B8E
:10C76000C4F85421274A21631268C4F8582194F868
:10C770003420C4F85C210023D4F88C20C4F8602154
:10C7800084F83430D4F88820C4F86421012384F874
:10C790006C3194F87431092B06D194F85C20022A8C
:10C7A00004BF052284F85C20D4F87821002A00F028
:10C7B000D680092B40F0D38094F85C30012B40F0F8
:10C7C000CE80216B1048002350F823508D4240F05A
:10C7D000C280052384F85C30C1E000BF0C80FF1FDD
:10C7E0006C96FF1F2896FF1F2893FF1F8397FF1F3C
:10C7F000F095FF1F3996FF1F0887FF1F7497FF1FD3
:10C800009097FF1F7496FF1FF487FF1F03A8FBF785
:10C8100085FF054600284ED0FBF798FF08B184F845
:10C82000A66194F8A6219DF80C10531CDBB222449B
:10C83000092B84F8A63182F8A7117FF422AF5E4A53
:10C8400094F8A71152780023914284F8A6317FF41E
:10C8500018AF5A495A5C01331644082BF6B2F9D185
:10C8600094F8AF31B34222D1554B94F8A8211A70F5
:10C8700094F8A9215A7094F8AA219A7094F8AB21DF
:10C880009A7194F8AC215A7194F8AD211A7194F808
:10C89000AE21DA70FBF7F0FE4A4B4B4A18600023DA
:10C8A0001370032284F8742184F8A63196E60423D9
:10C8B00084F87431E5E60AAE3046FCF796F948B3E1
:10C8C0002B46F25C01331544082BEDB2F9D19DF8EB
:10C8D0003020AA42ECD13A4B9DF829201A709DF8DD
:10C8E0002A205A709DF82B209A709DF82C209A715E
:10C8F0009DF82D205A719DF82E201A719DF82F2039
:10C90000DA70FBF7B9FE2F4B18602F4B00221A701C
:10C91000072361E694F85C30013B012B3FF6B1AE92
:10C92000236BB3F5C05F0CD2FCF73AF948B1206B2A
:10C930002349431C2363FCF794FA092384F87431D8
:10C9400053E6002384F85C309BE6D55401332F2B4B
:10C950007FF4F2AE1DE701339A427FF435AF0FB09A
:10C96000BDE8F08394F87401082804D840F251120D
:10C97000C240D207F3D4D4F87001144DD3F8033079
:10C980006970B0F5C05F6B6012D20D49FCF762FAB6
:10C990000B49D4F87001FCF788FA38B1D4F870313B
:10C9A0000133C4F8703165232B70D8E70723FBE708
:10C9B00007232B7000230DE70C80FF1F1F88FF1F2C
:10C9C0006C96FF1F3096FF1F3796FF1F8897FF1F3B
:10C9D000704710B5074CFBF74FFE2368C01AB0F53F
:10C9E000FA7F05D9044B0222DA60FBF745FE20608E
:10C9F00010BD00BF949BFF1F00F00F40704708B5AB
:10CA0000034B5878FCF774F8024B586008BD00BF20
:10CA10006C96FF1F8897FF1F7047704770477047DD
:10CA200070477047024B185C431F5842584170478B
:10CA30002888FF1F38B505460C46A1B901F05CFEF9
:10CA4000214620F4E072284601F030FE60236B435B
:10CA50001B4AD35C9BB328464FF000620721BDE818
:10CA6000384001F089BE002101F046FE04F00303C6
:10CA7000022B20F4E0721CD0032B1DD0012B01D11E
:10CA800042F04002630748BF42F4807214F0080489
:10CA900018BF42F400720021284601F007FE002C66
:10CAA000D9D128464FF000620721BDE8384001F097
:10CAB00071BE42F08002E5E742F0C002E2E738BD15
:10CAC000C494FF1F73B5144C23180646DB780D463B
:10CAD00023B94FF0C052072101F05CFE0F4A6023DA
:10CAE00003FB062301229B7D019285EAE572A2EBFE
:10CAF000E572D2B2009206210022304601F0ACFD70
:10CB0000002D04EB060304EB8604B4BF01220222CD
:10CB1000DA70A56002B070BD2888FF1FC494FF1FA3
:10CB2000184B1A1873B5D178044641B303EB800350
:10CB30000025D57007214FF080529D6001F01CFE4A
:10CB40004FF000620721204601F024FE60230E4AC8
:10CB50006343D618D35C93B15021204601F0CCFD3D
:10CB600021210246204601F0A1FD327DB37D0192D4
:10CB7000727D009206212A46204601F06DFD02B02A
:10CB800070BD00BF2888FF1FC494FF1F2DE9F34725
:10CB9000954D2C7D05F115084CB9E0B2FBF759FF16
:10CBA00008F804000134082CF7D101232B75DFF8B5
:10CBB0006CA28E4F272400264FF00209F0B2FBF73B
:10CBC00048FF18F80630834216D0B31D08F8060057
:10CBD0005AF82330022B0AD0032B02D0012B0BD1A1
:10CBE00050B13B5D012B08BF07F8049004E018B971
:10CBF0003A5D012A00D13B550136082E04F10104AB
:10CC0000DCD17B4CE369C3B17A4E3778AFB9FBF71F
:10CC100033FD794B1B68C01A0028E369B8BF404256
:10CC200098420AD9384601F0FDFD012001F0FAFDD5
:10CC3000022001F0F7FD01233370236AC3B16F4E68
:10CC40003778AFB9FBF718FD6D4B1B68C01A002889
:10CC5000236AB8BF404298420AD9384601F0E2FD43
:10CC6000012001F0DFFD022001F0DCFD0123337023
:10CC70002221687F634E01F03FFD0702687F01F0CB
:10CC8000B8FD0446687F642303FB00631B69002B27
:10CC900000F09C80002B87EAE772A2EBE772B8BF36
:10CCA0005B429A4240F392802B189B7F43B94FF02E
:10CCB0008062012101F060FD6B7F01222B449A7795
:10CCC00004F00903092B31D1687F4849C21C8B5CF1
:10CCD000DBB2012B0ABF4FF0020E8B5C01F802E0C1
:10CCE00049490A7818BFB3FA83F342FA00FE18BF25
:10CCF0005B091EF0010F15D04FF0010CDFF8208109
:10CD00000CFA00FE88F800E0DFF8188188F800C00F
:10CD1000DFF814C19CF800C0BCF1000F02D122EA78
:10CD20000E020A7013B1092101F070FDA2000CD5AA
:10CD3000687F2E4A00F10F03D15C012904BF022154
:10CD4000D1544FF0005101F061FD230505D527B9FD
:10CD50004FF40061687F01F059FDE00405D527B963
:10CD60004FF48051687F01F051FDA10405D527B92A
:10CD70004FF40051687F01F049FD620405D527B9E1
:10CD80004FF48041687F01F041FDFBF775FC6B6A51
:10CD9000C01A0028B8BF40420A287BDD687F1B4BC1
:10CDA0001B4A1C491C4F0344024401EB800101F063
:10CDB000E4FB6C7F2A5D6023052A51D8DFE812F07E
:10CDC00036006D00B500FB000D0150012B189B7F54
:10CDD000002B3FF475AF4FF08062012101F0DAFCC7
:10CDE0006B7F00222B446AE72888FF1F3996FF1FBC
:10CDF0000C80FF1F3796FF1F3096FF1F2893FF1FE1
:10CE00002896FF1F9493FF1F6093FF1F9093FF1FAF
:10CE10004C93FF1F6493FF1FC494FF1FF095FF1FE7
:10CE20005293FF1F6896FF1F3893FF1F6343FB5CFD
:10CE3000B3B1204600F03AFC90B91021204601F031
:10CE400095F8642303FB046620F4F852737ADB0838
:10CE500042EA03221021204601F042F801232B551B
:10CE6000687F00F093F96C7F60236343FB5C3BB108
:10CE70002B19DB78012B00F03F81022B00F0488159
:10CE80006B7F0133DBB2022B88BF00236B77FBF78C
:10CE9000F3FB686202B0BDE8F0870022052120465E
:10CEA00001F004FC602202FB04722046117D937D98
:10CEB0000191527D00920621002201F0CDFB7921E3
:10CEC000204601F019FC7F281BDCC0F180060422FB
:10CED0002021204601F0EAFB914A2421204601F05E
:10CEE000E5FB2121204601F007FC3721821920466D
:10CEF00001F0DCFBFBF7C0FB05EB84039862022327
:10CF0000ADE7B0F5C07F02DAC0F5C076DFE7B0F577
:10CF1000207F02DAC0F52076D9E7B0F5607FB4BF94
:10CF2000C0F56076C0F59066D1E7FBF7A5FB05EB91
:10CF300084039B6AC01A0028B8BF4042B0F57A7FCC
:10CF40008EDD642303FB0466F66956B12121204679
:10CF500001F0D2FB50210246204601F0A7FB03233B
:10CF60007DE732462021204601F0A0FB32462421F5
:10CF7000204601F09BFB5021204601F0BDFB212102
:10CF80000246204601F092FB2121204601F0B4FB2D
:10CF900037210246204601F089FB04222021204649
:10CFA00001F084FB5E4A2421204601F07FFB5D4BAB
:10CFB00001221A55D3E74FF0C0520721204601F055
:10CFC000E9FB594A0721204601F0D6FBFBF754FB49
:10CFD00005EB84039862042341E7FBF74DFB05EB67
:10CFE00084039B6AC01A0028B8BF4042B0F57A7F1C
:10CFF0007FF736AF4FF019420721204601F0CAFBF8
:10D00000642303FB0466737E0BB11B0725D54FF029
:10D0100020620721204601F0AFFB80220521204637
:10D0200001F044FB5921204601F066FB602303FB1D
:10D030000473002218613D4B5021204643F8242000
:10D0400001F05AFB21210646204601F055FB384BE2
:10D05000301A43F82400052301E74FF00072D8E7A7
:10D06000634317F80380B8F1000F7FF4F9AE204650
:10D07000FFF756FD4FF004620721204601F08AFBBE
:10D0800003220521204601F011FB642303FB046603
:10D090000621B37DB27A0193737A0093204643460A
:10D0A00001F0DAFA1021204600F060FF102140F470
:10D0B000F852204600F014FFF37D05F80480CBB948
:10D0C00001222021204601F0F1FA002224212046ED
:10D0D00001F0ECFA2121204601F00EFB134B53F82E
:10D0E00024202121821A204601F0E0FA0D4B012272
:10D0F0001A55B5E60222E4E75021204601F0FCFA79
:10D10000A0F5C332A03A2121204601F0CFFAB7E6BC
:10D110005021204601F0F0FA00F5C332A032F2E7C8
:10D1200040420F004F93FF1F000040814093FF1FBC
:10D130005493FF1F024B03EB80008068704700BFD1
:10D140002888FF1F38B5104A642303FB00230446D8
:10D15000DB7D0D46B3B90122202101F0A7FA20465C
:10D160004FF08052072101F007FB20464FF000628C
:10D17000072101F00FFB2A4620462421BDE8384054
:10D1800001F094BA0222E7E79493FF1F2DE9F84FCC
:10D190000F21C14D044601F0AFFA64236343E9183F
:10D1A0004FEA102B0A7A4F6812F0400F14BFEB5869
:10D1B00055F803904FEAD01016BF0BF0010A00F0AB
:10D1C000010A00F0010BA8461ABFC3F100097F4213
:10D1D0000BF0010B150602F03F06204612D501F0B8
:10D1E0002DFCB0FA80F04009731E072B00F2AC81D1
:10D1F000DFE813F00E000E000E000E003B013B01B5
:10D200003B013B0101F01AFC003018BF0120EBE7A5
:10D21000A24D2B5D013B0E2B00F29681DFE813F04F
:10D220000F001E002D003A004A00540063007100F8
:10D23000B200D900DF0094011D0127022202012162
:10D24000204601F059FA05EB840301225860023EA2
:10D25000934B96421A551BD8022333E005EB840307
:10D260005A6842F002020121204601F01FFA4946A5
:10D270002046FFF767FF032324E0BBF1000F00F017
:10D2800063812121204601F037FA864B43F82400C0
:10D29000042317E005EB84035A6842F001020121E0
:10D2A000204601F003FAC9F100012046FFF74AFFCA
:10D2B000052307E0BAF1000F00F04681204601F097
:10D2C000B1FA06232B553FE105EB840301215A688F
:10D2D000204622F0030201F0E9F939462046FFF723
:10D2E00031FF0723EEE7BAF1000F40F02D815146E0
:10D2F0002046FFF727FF79422046FFF723FF082348
:10D30000E0E7BAF1000F00F01F812121204601F073
:10D31000F3F9002106462046FFF714FF614A52F850
:10D3200024309B1B42F8243005EB840301215A680A
:10D33000204622F0030201F0B9F9642303FB0488BC
:10D3400098F81730E3B905222021204601F0AEF904
:10D350003A462421204601F0A9F94FF080520721D6
:10D36000204601F017FA4FF000620721204601F035
:10D3700003FA32463721204601F098F90923A1E744
:10D380000622E1E70F21204601F0B6F9C10740F17E
:10D39000DB802121204601F0AFF9434B00211860CA
:10D3A0002046FFF7CFFE00223721204601F07EF90C
:10D3B00000222121204601F079F95021204601F078
:10D3C0009BF9033E394B012E43F824004BD8794298
:10D3D000CDE0BAF1000F00F0B7800B2372E7BAF18D
:10D3E000000F40F0B1802121204601F085F951461F
:10D3F00006462046FFF7A6FE022396FBF3F605EB52
:10D40000840301215A68204622F0030201F04EF9FC
:10D41000642303FB048898F81730E3B90522202120
:10D42000204601F043F93A462421204601F03EF916
:10D430004FF080520721204601F0ACF94FF0006216
:10D440000721204601F098F932463721204601F0A5
:10D450002DF90D2336E70622E1E70F21204601F0E2
:10D460004BF9C20770D50E232CE70C4D2B5D013B09
:10D470000E2B69D8DFE813F01C002C003D004B0098
:10D480005C0068006A006800680092009C008000F0
:10D49000D100FB00F60000BF9493FF1F5C88FF1FC4
:10D4A0004F93FF1F2C93FF1FE495FF1F5493FF1F03
:10D4B000734B01212046195501F01EF905EB840339
:10D4C000062E58603FF4C8AE082E7FF4E1AEC3E6E6
:10D4D000062E05D105EB84035A6822F00302C0E64C
:10D4E000082E7FF4C4AE05EB84035A6822F00302D1
:10D4F000B9E6731F012B07D8BBF1000F04D0062E2D
:10D500003FF4C6AE0F23DDE6F0B10C23DAE6052EBC
:10D5100005D105EB84035A6822F00302BDE6072E0D
:10D520007FF4C1AE05EB84035A6822F00302B6E62D
:10D53000731F012B05D8BAF1000F02D0052EE1D1DF
:10D540008AE600287FF4CDAEBDE8F88F0028FBD135
:10D55000073E012E0AD905EB840301215A6822F007
:10D56000030242F00202204601F0A0F839462046AC
:10D57000FFF7E8FD0A23A5E60028E5D1073E012EC6
:10D580007FF625AF05EB840301215A6822F00302E0
:10D5900042F00102204601F089F818E70028D3D0B4
:10D5A0002121204601F0A8F805EB8403186114E757
:10D5B0000028C9D121212046A60001F09DF8AB1911
:10D5C00081465A68012122F00302204601F06EF8DC
:10D5D000642303FB048898F81730E3B9052220215F
:10D5E000204601F063F83A462421204601F05EF817
:10D5F0002E444FF080520721204601F0CBF84FF027
:10D6000000620721204601F0B7F8326991440222F6
:10D6100099FBF2F219E70622E1E70F21204601F01B
:10D620006BF8C30790D50E23212120462B5501F01E
:10D6300063F8144B002118602046FFF783FD002299
:10D640003721204601F032F800222121204601F046
:10D650002DF85021204601F04FF80B4B43F82400E1
:10D66000BDE8F88F00212046FFF76CFDFBE605EBD7
:10D67000840301215A68204601F018F8002321E6AE
:10D680004F93FF1FE495FF1F5493FF1F024B1A5C3B
:10D690000AB901221A5470475C88FF1F024B1A5CBA
:10D6A0000AB10F221A5470475C88FF1F014B185CA7
:10D6B000704700BF5C88FF1F0C4A116940F273235A
:10D6C0004B434FF6FF71B3FBF1F36E2B06D9084BBA
:10D6D0004FF4802159605723136070474F2B9EBF32
:10D6E000034B4FF480219960F5E700BF00B0034081
:10D6F00080F00F401B4B1A6802F01F02072A2ED839
:10D70000DFE802F0040B2D11171D23291A691649B1
:10D7100092B20A8041221A6070471A69124992B285
:10D720004A804322F7E71A690F4992B2CA8044221D
:10D73000F1E71A690C4992B20A814522EBE71A69AE
:10D74000094992B24A814622E5E71A69064992B22E
:10D750008A814722DFE71A69034992B2CA814022CF
:10D76000D9E700BF00B00B407888FF1F38B541F201
:10D770003001114B5A5842F000625A5041F23C01BC
:10D7800000245A5842F000625A5003F5E8230C2551
:10D7900040229D604920DC605C621A6001F07CF9E7
:10D7A000064B57229D602720DC605C621A60BDE852
:10D7B000384001F071B900BF0070044000B0034070
:10D7C0000B2829D8DFE800F0060A0D1028282828A1
:10D7D00013281E23114B188980B270470F4B5889AC
:10D7E000FAE70E4B9889F7E70C4BD889F4E70B4B17
:10D7F000588883B240F2732058434FF6FF7390FB72
:10D80000F3F07047054BD88883B28E20F4E7034BC2
:10D81000188883B24220EFE7002070477888FF1F06
:10D8200030B52E4D41F23C042B5943F010032B51DF
:10D830002B4B4FF400741C636FF4F8755C63A3F515
:10D840001433A4F13E542C441C604FF400545C602B
:10D85000244C1C601C68E401FCD50138072834D82E
:10D86000DFE800F0312F2D2B293327041E485860A4
:10D870001E4B002058631E4818601E484FF08064FD
:10D8800000EA8145C3F88040C3F88450FAB100EA49
:10D890008240C3F89040C3F894004FF08460C3F80E
:10D8A000A000C3F8A410AAB1C3F8B000C3F8B42014
:10D8B00030BD1148DBE71148D9E71148D7E71148D7
:10D8C000D5E71148D3E71148D1E71148CFE7C3F8AE
:10D8D0009020E2E7C3F8B02030BD00BF00700440E4
:10D8E000009004400F0080508720FE01004002405D
:10D8F0000F0080000000FC1F8720FE038720FE0F22
:10D900008720FE138720FE278720FE638720FEC71F
:10D910008720FE07384AD2F88030C3F30363022B16
:10D920005FD0D2F89030C3F30363022B5BD0D2F800
:10D93000A030C3F30363022B06D0D2F8B030C3F398
:10D940000363022B56D103231B0103F1402202F58E
:10D950000032D2F88010C1F303410170D2F8801078
:10D9600011F4801118BF01218170D2F8801011F4D8
:10D97000001118BF012141704178B1BBD2F8841069
:10D98000C1F38A4103F1402303F500334160D3F82A
:10D990008810090E0172D3F88810090C4172D3F86F
:10D9A0008810090A8172D3F88810C172D3F88C10DC
:10D9B000090E0173D3F88C10090C4173D3F88C1045
:10D9C000090A8173D3F88C30C373D2F880309B027C
:10D9D0004CBF4FF084634FF08063C2F88030012069
:10D9E00070470023B0E70123AEE7D2F8841021F09E
:10D9F0006041C7E70020704700400240184AD2F853
:10DA00007031C3F303630C2B10B527D044784368FF
:10DA100004B3C3F31103C2F874318368104A1BBA0C
:10DA2000C2F87831C3681BBAC2F87C318378002C05
:10DA300014BF4FF042624FF040620BB142F48012CB
:10DA400003781B0403F470231343054A0120C2F832
:10DA5000703110BD034901EA8343DCE7002010BDAB
:10DA6000004002400000FC1F0B4B4FF00062C3F867
:10DA700070214FF48022C3F87421084AC3F878213A
:10DA80006FF48471A2F166320A44C3F87C21044A1F
:10DA9000C3F87021704700BF00400240785634122E
:10DAA0000000080C10B53A4BDA7842F00202DA7046
:10DAB000384A1078C0B20228114641D0032835D028
:10DAC000012832D1546891688C4215D2D978C9079F
:10DAD00007D45168D0684C1C5460425CD2B21A71B1
:10DAE00010BD997801F0DF019970997801F0EF018C
:10DAF00099701074002317E0517C01F0FF0049B9C0
:10DB0000997801F0DF019970997801F0EF0199702F
:10DB1000107010BD997841F004019970917CC9B2E0
:10DB20001971002353740323137010BD997801F009
:10DB3000EF0199701B795169DBB20B700223F3E797
:10DB40009469D06984421DD2D2698869121A012A67
:10DB500005D19A7802F0DF029A7000230B70CB692E
:10DB60008A699B1A022B9FBF094A937843F00803E6
:10DB700093708A694869531C8B61054B1B79DBB232
:10DB8000835410BD997801F0DF019970B2E700BFAE
:10DB9000007006408C88FF1F41F234020A498B58FE
:10DBA00043F080038B50094B4FF418729A62DA628B
:10DBB00003F5E0331B225A70C0229A7000225A717A
:10DBC000192000F069BF00BF0070044000B004409D
:10DBD00010B5104B00241C745C749A6001225C60C8
:10DBE0001A700D4AD960917801F0F701917091781F
:10DBF00041F010019170917800F0FE0041F0200199
:10DC0000917010711A78002AFCD1187CB0FA80F05B
:10DC1000400910BD8C88FF1F0070064010B5104BE6
:10DC200000241C745C74DA6103229C611A700D4A32
:10DC30005961917801F0F7019170917841F01001EC
:10DC40009170917840F0010041F0200191701071C5
:10DC50001A78002AFCD1187CB0FA80F0400910BD77
:10DC60008C88FF1F0070064070B5144C002563615E
:10DC70000126049B25746674A2606560E36140EA36
:10DC80000603A561A3740E4BE16026709A7802F03A
:10DC9000F7029A709A7842F010029A709A7800F01F
:10DCA000FE0042F020029A7018712378002BFCD1FC
:10DCB000207CB0FA80F0400970BD00BF8C88FF1F47
:10DCC000007006402DE9F3411B4F1C4C00264FF01D
:10DCD0000C08F5B20423BA8FCDF800800A2128463B
:10DCE00000F066FD4FF480520021284600F0DEFC73
:10DCF000FA695421284600F0D9FC00225021284618
:10DD000000F0D4FC626CFF21082384F8401084F8F2
:10DD10004130019100936321D3B22846C2F3072218
:10DD2000013600F099FC032E07F1640704F160044A
:10DD3000CFD102B0BDE8F0819493FF1FC494FF1FC0
:10DD400038B50D460721044600F0D6FCEB074CBF62
:10DD500040F0800220F08002A8074CBF42F480729D
:10DD600022F4807269074CBF42F0100222F01002C8
:10DD70002B074CBF42F4007222F40072E8064CBF3D
:10DD800042F0040222F00402A9064CBF42F008024D
:10DD900022F008026B064CBF42F0200222F0200263
:10DDA00028064CBF42F0400222F04002E9054CBF79
:10DDB00042F0020222F00202AB0520464CBF42F4C0
:10DDC000806222F480620721BDE8384000F06EBC1A
:10DDD000072108B500F090FCC0F3C013C20548BF8E
:10DDE00043F00203C10648BF43F00403820548BF65
:10DDF00043F00803410748BF43F01003020748BF40
:10DE000043F02003810648BF43F04003420648BF69
:10DE100043F08003810748BF43F48073420548BF45
:10DE200043F40073184608BD2DE9F34701F07F075E
:10DE3000352F0546894692461C469DF828809DF858
:10DE40002C6016D143EA022448EA042446EA04245A
:10DE5000224A9F3024F4736424F0030452F82030E3
:10DE6000E404E40C23EA040442F8204002B0BDE8D4
:10DE7000F0876FF000720C2100F018FC0E2128468C
:10DE800000F03AFC4FF0FF320C21284600F00EFC67
:10DE900049F08003019300231A4600936D21284620
:10DEA00000F0DAFB0196CDF80080234652466C2143
:10DEB000284600F0D1FB0E21284600F01DFC83010E
:10DEC000F9D544EA0A2407EB470048EA0424284429
:10DED000024B46EA042443F82040C7E7AC88FF1F02
:10DEE000F7B501F07F05352D04460F4616460FD1D4
:10DEF0001D4A9F3426F4736626F0030652F8243038
:10DF0000F604F60C23EA060342F8243003B0F0BD11
:10DF10006FF000720C2100F0C9FB0E21204600F0CA
:10DF2000EBFB4FF0FF320C21204600F0BFFB47F027
:10DF3000800700231A466D2120460197009300F0C8
:10DF40008BFB32466C21204600F0B0FB0E212046B0
:10DF500000F0D2FB8301F9D505EB45052C44024BBB
:10DF600043F82460D2E700BFAC88FF1F73B51F4B96
:10DF700001F07F0405461B5D83B36FF000720C2136
:10DF800000F094FB0E21284600F0B6FB00264FF06F
:10DF9000FF320C21284600F089FB32466D212846CD
:10DFA00001940096334600F057FB32466C21284618
:10DFB00000F07CFB0E21284600F09EFB8201F9D583
:10DFC0006E21284600F098FB222C01D0422C03D170
:10DFD000030201D540F07F4002B070BD04EB440461
:10DFE0000444034B53F82400F6E700BFA4160100D5
:10DFF000AC88FF1F70B50B4C2218054692F800261E
:10E000000E465AB96C21FFF7B1FF06F00F0320F05E
:10E010000F021A436C212846FFF762FF631983F849
:10E02000036670BDAC88FF1F38B50C466C210546F1
:10E03000FFF79CFF240104F0700420F070022243DB
:10E0400028466C21BDE83840FFF74ABF38B50C467A
:10E050006C210546FFF78AFFE40304F4C03420F482
:10E06000C032224328466C21BDE83840FFF738BF54
:10E0700038B50C466C210546FFF778FF240504F4FB
:10E08000700420F47002224328466C21BDE8384019
:10E09000FFF726BF38B50C466C210546FFF766FF33
:10E0A000240604F0706420F07062224328466C213C
:10E0B000BDE83840FFF714BF38B50D466C21044663
:10E0C000FFF754FF3DB140F0804220466C21BDE88F
:10E0D0003840FFF705BF20F08042F6E738B50D461F
:10E0E0006C210446FFF742FF3DB140F40022204678
:10E0F0006C21BDE83840FFF7F3BE20F40022F6E7BC
:10E1000038B50D466C210446FFF730FF3DB140F4B1
:10E11000802220466C21BDE83840FFF7E1BE20F4A4
:10E120008022F6E738B50D466C210446FFF71EFF46
:10E130003DB140F4804220466C21BDE83840FFF7F5
:10E14000CFBE20F48042F6E738B50D466C21044678
:10E15000FFF70CFF3DB140F4005220466C21BDE8B2
:10E160003840FFF7BDBE20F40052F6E738B50D4643
:10E170006C210446FFF7FAFE3DB140F48052204680
:10E180006C21BDE83840FFF7ABBE20F48052F6E7C3
:10E1900038B50C466C210546FFF7E8FE230748BF5B
:10E1A00020F070004FEA04124CBF40F4006020F4ED
:10E1B000076002F0700202436C212846BDE8384037
:10E1C000FFF78EBE38B50C466C210546FFF7CEFE34
:10E1D000E40104F4F06420F4F062224328466C2148
:10E1E000BDE83840FFF77CBEFFF7ECBF38B50D4601
:10E1F0006C210446FFF7BAFE3DB140F400322046E0
:10E200006C21BDE83840FFF76BBE20F40032F6E722
:10E2100008B5074B034493F800262AB96C21FFF791
:10E22000A5FE00F00F0008BD93F8030608BD00BF6F
:10E23000AC88FF1F08B56C21FFF798FEC0F30210F1
:10E2400008BD08B56C21FFF791FEC0F3C13008BDD1
:10E2500008B56C21FFF78AFEC0F3035008BD08B56E
:10E260006C21FFF783FEC0F3036008BD08B56C2185
:10E27000FFF77CFEC0F3807008BD08B56C21FFF786
:10E2800075FEC0F3C04008BD08B56C21FFF76EFEF7
:10E29000C0F3804008BD08B56C21FFF767FEC0F3EE
:10E2A000803008BD08B56C21FFF760FEC0F3403038
:10E2B00008BD08B56C21FFF759FEC0F3003008BD5A
:10E2C00008B56C21FFF752FEC0F30213020548BFE8
:10E2D00043F00803184608BD08B56C21FFF746FE59
:10E2E000C0F3C31008BDFFF7F7BF08B56C21FFF7F7
:10E2F0003DFEC0F3404008BD38B50C466D210546D3
:10E30000FFF734FE640104F0600420F06002224351
:10E3100028466D21BDE83840FFF7E2BD38B50C4610
:10E320006D210546FFF722FE640304F4C04420F487
:10E33000C042224328466D21BDE83840FFF7D0BDDA
:10E3400038B50C466D210546FFF710FE240204F493
:10E35000706420F47062224328466D21BDE8384085
:10E36000FFF7BEBD38B50C466D210546FFF7FEFD33
:10E3700004F00F0420F00F02224328466D21BDE86F
:10E380003840FFF7ADBD38B50D466D210446FFF7A7
:10E39000EDFD20F47F0040EA05426D212046BDE8F6
:10E3A0003840FFF79DBD38B50D466D210446FFF797
:10E3B000DDFD3DB140F4004220466D21BDE838400E
:10E3C000FFF78EBD20F40042F6E738B50D466D210B
:10E3D0000446FFF7CBFD3DB140F0807220466D2131
:10E3E000BDE83840FFF77CBD20F08072F6E708B545
:10E3F0006D21FFF7BBFDC0F3411008BD08B56D21CD
:10E40000FFF7B4FDC0F3413008BD08B56D21FFF73B
:10E41000ADFDC0F3032008BD08B56D21FFF7A6FDD3
:10E4200000F00F0008BD08B56D21FFF79FFD031434
:10E43000D8B21B0648BF60F0FF0008BD08B56D21CB
:10E44000FFF794FDC0F3C03008BD08B56D21FFF79C
:10E450008DFDC0F3006008BD38B50C46702105463F
:10E46000FFF784FD04F0030420F4401242EA045252
:10E4700028467021BDE83840FFF732BD38B50D465B
:10E4800070210446FFF772FD3DB140F400222046A2
:10E490007021BDE83840FFF723BD20F40022F6E7E5
:10E4A00038B50D4670210446FFF760FD3DB140F4DC
:10E4B000802220467021BDE83840FFF711BD20F4CE
:10E4C0008022F6E738B50C4670210546FFF74EFD71
:10E4D00004F0030420F4403242EA0442284670214A
:10E4E000BDE83840FFF7FCBC38B50D467021044646
:10E4F000FFF73CFD20F47F4040EA052270212046D2
:10E50000BDE83840FFF7ECBC38B50D467021044635
:10E51000FFF72CFD20F0FF0045EA000270212046A5
:10E52000BDE83840FFF7DCBC08B57021FFF71EFDE1
:10E53000C0F3015008BD08B57021FFF717FDC0F307
:10E54000C04008BD08B57021FFF710FDC0F3804042
:10E5500008BD08B57021FFF709FDC0F3014008BDF3
:10E5600008B57021FFF702FDC0F3072008BD08B50C
:10E570007021FFF7FBFCC0B208BD70B50E466C21E0
:10E5800015461C4600F0B8F816B1C0F349233360B5
:10E5900015B1C0F304432B700CB1000E207070BD98
:10E5A0002DE9F341FAF768F80446FAF765F8001B1D
:10E5B0000028B8BF40420928F7DD154E0024A046C8
:10E5C000F71EE5B24FF4803200212846FFF788FCA1
:10E5D000022255238DE80C006C21032300222846DB
:10E5E000FFF722FC1F230193009300231A461021FA
:10E5F0002846FFF719FC2846FFF70AFE04F80780B3
:10E6000030550134032CDCD102B0BDE8F08100BFED
:10E61000AF8EFF1F38B5074C044494F8001641B97B
:10E6200094F80356FFF7E6FC012384F8003684F8DB
:10E63000035638BDAC88FF1F064B034493F80026F1
:10E6400032B1002293F8031683F80026FFF7D2BCFC
:10E65000704700BFAC88FF1F2DE9F0411F46124BE9
:10E660009DF8186033F810409DF81C50904641F01A
:10E67000800100222046FAF723FB41460022204673
:10E68000FAF71EFB394600222046FAF719FB3146FD
:10E6900000222046FAF714FB294620460122BDE855
:10E6A000F041FAF70DBB00BF4C80FF1F38B5114B8E
:10E6B00033F81040154641F0800100222046FAF759
:10E6C000FFFA290E00222046FAF7FAFAC5F30741AD
:10E6D00000222046FAF7F4FAC5F30721002220466B
:10E6E000FAF7EEFAE9B220460122BDE83840FAF71F
:10E6F000E7BA00BF4C80FF1F38B51E4B33F81040FF
:10E70000002220460D46FAF7DBFA00221146204689
:10E71000FAF7D6FA002211462046FAF7D1FA00227B
:10E7200011462046FAF7CCFA012200212046FAF7DA
:10E73000C7FA294600222046FAF7C2FA00221146FB
:10E740002046FAF7BDFA0022114605022046FAF7E4
:10E75000B7FA0022114605432046FAF7B1FA2D0216
:10E760000543012200212046FAF7AAFA2D02284388
:10E7700038BD00BF4C80FF1F70B504460D461646DD
:10E78000FFF7BAFF294640EA06022046BDE870407E
:10E79000FFF78CBF70B504460D461646FFF7ACFF79
:10E7A000294620EA06022046BDE87040FFF77EBFFA
:10E7B0002DE9F8439DF8209098460F4606461446EA
:10E7C0000025FFF799FFC1444146012349450BD37A
:10E7D00004FA08F444402C4080EA040239463046EA
:10E7E000BDE8F843FFF762BF03FA01F215430131B8
:10E7F000ECE710B50C2104464FF0FF32FFF756FF4F
:10E8000020460E21BDE81040FFF776BF10B5CA4381
:10E8100004460C21FFF74AFF20460E21BDE81040B8
:10E82000FFF76ABF10B5084BC4B201221A54202169
:10E8300020460022FFF73AFF204600222421BDE8AF
:10E840001040FFF733BF00BF4F93FF1F2DE9F74381
:10E850000027714E714DDFF8CC91B846FCB24FF4F1
:10E86000805200212046FFF721FF4FF005121021B2
:10E870002046FFF71BFF4A4604212046FFF716FFFC
:10E880006FF000720C212046FFF710FF0E2120468A
:10E89000FFF732FF00231A466D212046CDF8048091
:10E8A000CDF80080FFF7D8FE00226C212046FFF74C
:10E8B000FDFE032205212046FFF7F8FE0422202159
:10E8C0002046FFF7F3FE002237212046FFF7EEFE39
:10E8D000002221212046FFF7E9FE4FF448022421BF
:10E8E0002046FFF7E3FE4FF4483228212046FFF789
:10E8F000DDFE4FF4483229212046FFF7D7FEB37DD5
:10E900000193737AB27A0093062100232046FFF721
:10E91000A3FEB38A424A15215A432046FFF7C6FE9A
:10E920006A6860212046FFF7C1FEAA68612120467F
:10E93000FFF7BCFEEB892A7B1C2143EA02422046FA
:10E94000FFF7B4FE2A6959212046FFF7AFFE2A6A75
:10E950005A212046FFF7AAFE6A6A5B212046FFF78C
:10E96000A5FEAA6A95F82C30D1B2C2F30722019114
:10E9700000925D2100222046FFF76EFE2A6B5E2189
:10E980002046FFF793FEAA6918212046FFF78EFE66
:10E99000EA6919212046FFF789FE6A6B5C2120464F
:10E9A000FFF784FEAA6B5F212046FFF77FFEEA6B2C
:10E9B00052212046FFF77AFE6A6C95F840300193A9
:10E9C00095F8413000936321D3B22046C2F3072269
:10E9D000FFF742FE95F84830CDF8048000227D21F3
:10E9E0002046CDF80080FFF737FE4FF4403201217A
:10E9F0002046FFF75BFE01376FF0004235212046CD
:10EA0000FFF754FE032F06F1640605F160057FF45D
:10EA100025AF03B0BDE8F0839493FF1FC494FF1F9C
:10EA2000007102008D123083034B10229A6000BFE8
:10EA300000BF00BF5A60704700F00F4008B50F21BB
:10EA4000FFF75AFEC0F3003008BD00027047800097
:10EA5000704700127047801070477047FEE74FF014
:10EA6000E0210B4A0B4BC1F8083D4CF22053D381F7
:10EA70004DF62813D381138823F001031B041B0CCC
:10EA80001380D1F8883D43F47003C1F8883D704786
:10EA90000020054000800000802800F01F014FF09A
:10EAA00001030F4A04DD8B40C2F88C31D3607047FC
:10EAB000402804DD8B40C2F88831936070472028DD
:10EAC00004DD8B40C2F8843153607047404200F04F
:10EAD0001F0058BF41428B40C2F88031136070471D
:10EAE00000E100E0802800F01F024FF001030D4913
:10EAF00003DD9340C1F88C307047402803DD93401C
:10EB0000C1F888307047202803DD9340C1F8843075
:10EB10007047404200F01F0058BF42429340C1F886
:10EB20008030704700E100E0074B1A78D2B2012A2A
:10EB300002D1222903D15A7001225A70704721292B
:10EB4000FAD10022F7E700BFB28EFF1F70B515465D
:10EB500011B91B4B197070BD022903D1184B01224A
:10EB60001A7070BD04291AD1154B5B78012B25D181
:10EB70009488402C28BF402400235E1CDBB2A342B3
:10EB800007D300231A4602211846BDE8704000F062
:10EB900047BF2A68D05C00F0C3F83346EDE703298D
:10EBA00006D1074A5378012B08D100239370E9E777
:10EBB000052901BF024B00221A705A7070BD00BFB8
:10EBC000B28EFF1F10B50446204600F0C1F80028A1
:10EBD000FAD110BD704738B50A4C012502460B46E4
:10EBE00000202946A57000F0F5FA224618B100234E
:10EBF000A370122038BD937803F0FF00002BFAD1E8
:10EC000038BD00BFB28EFF1FF8B506460F4600F0B4
:10EC1000F4FC0E4B1A78012A16D15B78012B13D124
:10EC200000F000F988B10025ECB2A74205D82146D2
:10EC30003046BDE8F840FFF7CEBF301900F0D6F8F7
:10EC400001350028F0D0F2E70C20F8BDB28EFF1F8E
:10EC500008B540210248FFF7D7FF00F095F808BD3E
:10EC6000B58EFF1F38B5054600F0A8F80B280446FE
:10EC700009D140210548FFF7C7FF28B92846BDE85C
:10EC8000384000F09BB80024204638BDF58EFF1FA9
:10EC900070B50C46461E00250CB9284670BD16F806
:10ECA000010FFFF7DFFF013C002818BF0B25A4B2BE
:10ECB000F2E738B5451E002415F8010F08B92046C3
:10ECC00038BDFFF7CFFF002818BF0B24F4E707B5C6
:10ECD0000123002200930649064B104600F020FA5B
:10ECE000002814BF1B20002003B05DF804FB00BF08
:10ECF0004DEB000029EB000038B50C46054600F04E
:10ED000097F8A0420AD32C440020A54207D000B1B6
:10ED100038BD15F8010B00F051F8F6E70B2038BDAF
:10ED200010B50A4A117840290ED05378D41801330F
:10ED3000DBB2402BA07001F101014FF00000117017
:10ED400014BF5370507010BD0B2010BD358FFF1FC6
:10ED500010B50C4A117891B192F84230D4180133B1
:10ED6000DBB2A4780470402B4FF0000001F1FF31BA
:10ED7000117014BF82F8423082F8420010BD0A20A0
:10ED800010BD00BF358FFF1F014B1878704700BFC3
:10ED9000358FFF1F024B1878C0F14000C0B270479A
:10EDA000358FFF1F034B00225A7083F842201A70E0
:10EDB000704700BF358FFF1FFFF7F4BF10B50A4A39
:10EDC000117840290ED05378D4180133DBB2402B90
:10EDD000A07001F101014FF00000117014BF5370D9
:10EDE000507010BD0B2010BD788FFF1F10B50C4A5E
:10EDF000117891B192F84230D4180133DBB2A47883
:10EE00000470402B4FF0000001F1FF31117014BF6E
:10EE100082F8423082F8420010BD0A2010BD00BFC7
:10EE2000788FFF1F014B1878704700BF788FFF1F46
:10EE3000024B1878C0F14000C0B27047788FFF1FB6
:10EE4000034B00225A7083F842201A70704700BFAB
:10EE5000788FFF1FFFF7F4BF70B50546007801F00B
:10EE600093F902780023D9B2914207D25C1C03EBDC
:10EE7000830303445E786B789E4227D1174C2B7A2C
:10EE8000342202FB0142D67813B334234B43E218F9
:10EE9000907886420CD000F0030204330C2010FB63
:10EEA00002302118205C0B894A68497800F090FBF9
:10EEB000D4F89C3083B12A46287812F8081F00291C
:10EEC0000CBF03210521BDE8704018472346CAE75F
:10EED000937801339370D8E770BD00BFBC8FFF1FDC
:10EEE0002DE9F04F85B00D4690468DF80F0001F0EA
:10EEF0004BF9022D064647D1077800235C1CDBB294
:10EF0000BB4210DB4FF00009DFF8B0B0CA465FFA31
:10EF100089F4A74212DC284BD3F89C30002B45D152
:10EF200005B0BDE8F08F03EB830333440DF10F0010
:10EF3000DA78597801F0E2F92346DFE704EB84043C
:10EF40003444E378A2886178CDF804A0A0780090DA
:10EF50000DF10F0001F0B0F9A378032B05D15A464B
:10EF600061789DF80F0001F031FA6178E37841F0A3
:10EF7000100141EAC3110022C9B20DF10F0001F0E6
:10EF8000EDF909F10109C2E7002DC4D10A4903785E
:10EF9000342000FB03138A1C3633294634329A424C
:10EFA000B9D002F8341C02F8331CF7E74246294670
:10EFB0009DF80F009847B3E7BC8FFF1F59EE000084
:10EFC000F0B40C7804F06004202C1D4632D14C784B
:10EFD000042C1DD00AD8012C04D003D3022C20D03D
:10EFE000032C12D000202880F0BC7047212C1BD0AD
:10EFF00004D8202CF6D1F0BC00F040B9222C16D059
:10F00000232CEFD1F0BC00F049B9F0BC00F049B9B5
:10F0100002241C801468002525701468671C176082
:10F020006570F0BC00F056B9F0BC00F01FB9F0BC40
:10F0300000F076B9402C06D1044CD4F8A04014B1AD
:10F04000A446F0BC6047CD20CEE700BFBC8FFF1FB9
:10F0500073B50446007801F097F863680093A27ACC
:10F06000637A43EA0223ADF8043002780023D9B270
:10F07000914207D25D1C03EB830303445E786378FF
:10F080009E4225D1174D237A342202FB0152D678B5
:10F0900003B334234B43EA18907886420CD000F037
:10F0A000030204330C2010FB02302918285C0B8962
:10F0B0004A68497800F08CFAD5F89C3033B1227A4E
:10F0C00020785AB104F108020521984702B070BDBA
:10F0D0002B46CCE7937801339370DAE76A46032135
:10F0E000F3E700BFBC8FFF1F07B543680093437A67
:10F0F000817A43EA0123ADF80430084BD3F89C3001
:10F1000002462BB1017A007829B1083205219847CF
:10F1100003B05DF804FB6A460421F8E7BC8FFF1FCB
:10F120002DE9F84305460F461646984601F02CF89F
:10F1300002789DF8203001328146D2B20021284663
:10F1400001F09EF80446E8B9164A1749284600F02F
:10F1500086F999F80000154B342200FB022209F1D0
:10F1600001011A4499463433934201F105010CD14F
:10F170004146284600F074F8044618B9C9F89C7056
:10F18000C9F8A0602046BDE8F88311F8050C03F823
:10F19000340C11F8040C03F8330C03F8324C03F868
:10F1A000314CE0E7C1EF0000E1EE0000BC8FFF1F33
:10F1B00008B5074B0022C3F89C20C3F8A02000F03C
:10F1C000A1F918B9BDE8084001F06EB808BD00BF4C
:10F1D000BC8FFF1F2DE9F041984605460E461746A5
:10F1E00000F0D2FF04780023D9B2A14207D2013344
:10F1F00003EB8302024412F8042CB242F4D1174C00
:10F2000034234B43E218D07892F802E0A0EB0E01D1
:10F21000C9B2042902D1C120BDE8F08100F0030188
:10F220000130C0B24FF00C0C0CFB0133D070A0EBDE
:10F230000E001C44C0B2012825716671A760A4F8B5
:10F240000C8007D143463A4631462846BDE8F04196
:10F2500000F0BEB90020BDE8F08100BFBC8FFF1FE9
:10F26000014B0020196070476090FF1F024B097925
:10F27000197100F08DBF00BF6090FF1F13B500240F
:10F2800002AA1C80044B42F8041D0979197100F090
:10F290008DFF02B010BD00BF6090FF1F00201880DE
:10F2A000704730B40C460221198021796488084DDA
:10F2B000012C297102D130BC00F08EBF022C02D18A
:10F2C00030BC00F095BF0020188030BC704700BFF4
:10F2D0006090FF1F30B40C460221198021796488A8
:10F2E000074D012C297102D130BC00F08DBF022CDA
:10F2F00002D130BC00F09ABF0020188030BC7047AB
:10F300006090FF1F044B054A19795B7911711372E4
:10F3100003210A23FFF75EBF6090FF1F5280FF1F8B
:10F32000F8B500271F808B780B4CA371C3F3400303
:10F330005A0063F3000206466271FFF7E3FF256897
:10F3400045B1A37913F002021ABF3A4622212121C6
:10F350003046A8470020F8BD6090FF1F034B00F126
:10F3600008021B6800780521184700BF6890FF1F3E
:10F3700070B5094D04462A1D012100F0D7FF8022F7
:10F380000121204600F0EAFF2B68207800220A21A4
:10F39000BDE87040184700BF6890FF1F37B50121D6
:10F3A0000DF10702044600F0C1FF9DF80730074D3C
:10F3B000802B04D12A790121204600F0CFFF2B6851
:10F3C000207800220B21984703B030BD6890FF1FC2
:10F3D000436805215A7800F0C1BF73B501220024AB
:10F3E00005460126002100F089FF334621468DE8BD
:10F3F00050001022284600F05FFF22462146284692
:10F4000000F07CFF234621468DE85000102228465C
:10F4100000F052FF31460222284600F09FFF32469C
:10F420000621284600F09AFF22469021284600F047
:10F4300095FF044B28781B682246214602B0BDE8A0
:10F44000704018476890FF1F42783AB9C178C901E7
:10F4500041F0100101F0900100F080BF704773B5DA
:10F460000C468DF8070001F00DFA1F4D2C60044684
:10F47000002836D11D4A9DF80700102100F0A6FF94
:10F480001B4A044612219DF8070000F09FFF194A0D
:10F49000044314219DF8070000F098FFE4B20443F0
:10F4A000154A9DF80700132100F090FFE4B20443D1
:10F4B000124A9DF80700172100F088FF02AEE4B25F
:10F4C00004430F4A16F8010D162100F07FFFE4B245
:10F4D000044303220121304600F040FF0323E4B23D
:10F4E0002B71204602B070BD6890FF1FDBF3000057
:10F4F000D1F3000071F300009DF3000049F4000017
:10F500005DF3000037B502AD174B05F8010D002281
:10F51000102128461A6000F05BFF1221044628469D
:10F5200000F056FF14210443284600F051FFE4B2D6
:10F5300004431321284600F04BFFE4B20443172193
:10F54000284600F045FFE4B204431621284600F0A7
:10F550003FFFE4B2204310F0FF0003D19DF8070005
:10F5600001F09CF903B030BD6890FF1F1FB5012169
:10F570008DF807000DF10E020DF1070000F0D6FE28
:10F580000DF10F0206210DF1070000F0CFFE9DF8EE
:10F590000E30802B18D19DF80F309B0714D59DF8A5
:10F5A000070000F0EFFD012804460DD172B60DF101
:10F5B000070000F029FB002221460DF107008DF81D
:10F5C0000E2000F0CBFE62B69DF80E0004B010BD18
:10F5D00073B50C4615461E468DF80700FFF7C6FFAB
:10F5E000802808D033462A4621460DF1070000F056
:10F5F000A7FA02B070BD0020FBE77047062812D8BA
:10F6000080000129C0B201D10230C0B2074AC0F364
:10F610004703122101FB03231A884FF6FF739A4216
:10F6200008BFFF207047FF20704700BF7090FF1F8A
:10F630002DE9F041314C324D324E4FF0000884F844
:10F6400000814FF4107285F840020F462846FF21D2
:10F6500001F0D0FE4FF4806241463046C5F8446266
:10F6600001F0C8FE94F80C3143F0800384F80C31AB
:10F6700094F80C311B06FBD4234BFF221A7094F82C
:10F680000C3143F0400384F80C31204B196897B3D8
:10F6900041F000411960194B310AC6F3074201F0ED
:10F6A000FE0183F89C1083F8B020320E83F8B4205A
:10F6B000174AC5F84822102283F80821012283F84E
:10F6C0009420BF2283F8802093F8002102F07F026B
:10F6D00083F8002193F8842042F0010283F884200B
:10F6E00093F8842042F0100283F8842084221A7751
:10F6F0000020BDE8F08121F00041CBE70020074069
:10F700007090FF1F009CFF1F5C80FF1F0070044073
:10F71000009EFF1F0D4B93F80C2102F0BF0283F8EF
:10F720000C21BF2283F8802093F8842002F0FE028F
:10F7300083F8842093F8942002F0FE0283F894204A
:10F740001A7F02F07B021A770020704700200740E2
:10F75000F7B5082304248DE81800B1F803300D78BC
:10F760008878B3F5007F81BF0023CB7002230B7133
:10F77000062D71D8AB00DCB2012804BF0234E4B21C
:10F780004FEA540E354C122707FB0E474FF6FF7613
:10F79000B7F800C0B4455FD14E78032E5CD801287D
:10F7A0005AD897F80FC0BCF1FF0F04BF4FF0000C00
:10F7B00087F80FC0B1F803C0122101FB0EFE04EB65
:10F7C0000E0743EA4003BA73FA7B7E7402F001022B
:10F7D00013435BB2D4F84822C7F80220D9B2F973B8
:10F7E0003874D4F8447224F80EC01BB207EBC30E71
:10F7F00081F00101CEF80420AEF802C04FF0080EEF
:10F8000007F833E007EBC10ECEF80420AEF802C0D3
:10F8100012FA8CF24FF0480E07F831E0C4F8482293
:10F8200028B917F8332062F07F0207F8332002AAC4
:10F8300002EB80002DB20A4950F8082C11F825304F
:10F84000012E0CBF164642F001063343DBB201F82D
:10F850002530002003B0F0BD9520FBE77090FF1F1E
:10F86000C0200740084610B51146FFF7C7FEFF2825
:10F870001DD0104B1221C0F3470001FB0030D3F81C
:10F880004422C37B1CB283F0010312F8341001F050
:10F890007F0102F8341012F8331001F07F0102F8F2
:10F8A00033104FF0FF338372C372002010BDC420A9
:10F8B00010BD00BF7090FF1F73B50C468DF8070098
:10F8C000114620461646FFF799FEFF28054620D030
:10F8D000214632460DF10700FFF7C4FFC5F3470389
:10F8E00012210D4D59436B18D5F848221888121A69
:10F8F000C5F8482224B2094A002002F824004FF03B
:10F90000FF326A549A705A70DA701A715A7102B0E2
:10F9100070BD9620FBE700BF7090FF1FC02007401E
:10F920002DE9F0410E468046114630461746FFF756
:10F9300065FE0C4DC0F34700122303FB0050C47B4F
:10F94000FF2C0DD03A4631464046FFF78BFF24B2DC
:10F95000D5F8442212F8343063F07B0302F83430D7
:10F96000BDE8F0817090FF1F10B5084600211446D5
:10F97000FFF744FE084AC0F34700122101FB0020B4
:10F98000D2F84432C27B03EBC2035A681368236087
:10F990005368636010BD00BF7090FF1F10B50C4628
:10F9A00020461146FFF72AFEFF281AD024B2104B3A
:10F9B00013F82430DBB213F00C0F12D09B0712D4D3
:10F9C0000C4BD3F8443213F83020D2090DD180F01B
:10F9D0000100C0B213F83030DB0914BF032000204F
:10F9E00010BD052010BD012010BD032010BD00BFBB
:10F9F000C02007407090FF1F08B5FFF7FFFD074AC2
:10FA00001223C0F3470003FB0020C37BFF2B1EBF64
:10FA1000D2F84422002102F8331008BD7090FF1F75
:10FA20002DE9F0410846002190461F46FFF7E6FD0C
:10FA30002249C0F34700122404FB0014E57BFF2D8C
:10FA400039D022884FF6FF7093B2834233D0D1F879
:10FA5000441285F0010011F9300000282BDB2EB292
:10FA600087B901EBC60338465A80D4F802205A60A1
:10FA700011F8352002F0400262F0770201F83620DA
:10FA8000BDE8F08101EBC602BB424FF0000028BF89
:10FA90003B466781C4F80680207360735380C2F8C8
:10FAA000048011F8353003F0400363F0770301F868
:10FAB0003630BDE8F0819420BDE8F0817090FF1FE2
:10FAC0002DE9F0410C460646114620461546FFF743
:10FAD00095FD194BC0F34700122202FB003090F84D
:10FAE0000FE0BEF1FF0F24D027B2144A6CB1407C66
:10FAF000012D0CBF14211821012818BF41F001016C
:10FB000012F82700014302F8271012F827106FF3AC
:10FB1000410102F82710D3F84432002203F83E20B6
:10FB20003DB92B462A4621463046BDE8F041FFF755
:10FB300077BFBDE8F08100BF7090FF1FC020074075
:10FB40002DE9F0410C462046012117469846FFF763
:10FB500055FDFF2836D01C4BC0F34700122202FB94
:10FB60000030D3F8446290F80FE016F93E30002BD5
:10FB700028DB23B2154A12F8235015F0020521D1D3
:10FB80000188C0F806701FFA88F242818A42D8BF05
:10FB900011460FFA8EF206EBC203057345735980C6
:10FBA0005F602CB9C82306F832302046BDE8F081EA
:10FBB00016F83E3003F0400363F0770306F8323066
:10FBC0002C46F2E79324F0E77090FF1FC020074017
:10FBD000034B044883F898100122114600F0BEBB85
:10FBE00000200740B092FF1F054B0648002283F813
:10FBF0009420802283F80C210121FF2200F0AEBB6B
:10FC000000200740B092FF1F38B51A4C94F800212D
:10FC100002F07F0284F8002194F80C2102F0DF0248
:10FC200084F80C2194F8802042F0200284F880208F
:10FC300094F8842002F0DF0284F8842094F8942061
:10FC400002F0DF0284F8942094F8942042F0040239
:10FC500084F8942044F62065013DADB200F0BCFE6E
:10FC6000002DF9D194F8943003F0FB0384F894301C
:10FC700038BD00BF002007402DE9F04FD84DD94CCA
:10FC800095F8807095F8843095F8906087B0FF22E1
:10FC90001F4094F840328DF809208DF80C308DF813
:10FCA0000D20002301210DF1090204F510708DF8DB
:10FCB0000E3004938DF815308DF816308DF80F3016
:10FCC0008DF8143000F032FB95F80C31D907F6B2FC
:10FCD0000FD59DF80930802B0BD195F8003103F03A
:10FCE0007F0385F8003195F80C3103F0DF0385F8C8
:10FCF0000C317A0711D5BA4B042093F8A41093F86D
:10FD0000A02083F8800006AB42EA012223F80E2DE2
:10FD100003A91220049300F06DFBFB074BD5B04DF7
:10FD2000B0480123BF2685F8803085F8886095F8B3
:10FD30009430002743F0020385F894304FF410729A
:10FD400085F89870FF2185F8007101F053FB4FF49E
:10FD500080623946D4F8440201F04CFBD4F84432B6
:10FD600003F50073C4F848329F4BFF221A7095F8D0
:10FD7000943003F0FD0385F8943095F80C3143F08E
:10FD8000400385F80C319F2385F88C6085F884301A
:10FD900095F8943003F0DF0385F8943003A9102020
:10FDA00000F028FB95F8943003F0DF0385F89430D9
:10FDB00007B0BDE8F08F3D0740F19380884B0822E3
:10FDC00083F880203309C6F3C000062B8DF80D3070
:10FDD0008DF80F0000F2F480C6F3800202EB83027C
:10FDE00008B10232D2B2D4F8446206EBC201C2F3C7
:10FDF0004705D1F804E04988ADF81510122101FB40
:10FE00000541CDF810E091F80FC08CF0010C81F89D
:10FE10000FC016F8321082F0010A5FFA8AFAC1F3B5
:10FE200080110FFA8AF881F00101890106EBC809F7
:10FE300006F83810002800F0D980DFF8ACB19BB983
:10FE40009BF8002082B9FF2219468BF8002003A8F6
:10FE50001A460193FFF706FD019B06F838301A4653
:10FE6000194603A8FFF7DCFD9BF80030012B04D0F6
:10FE70009DF80D30002B00F0AD80122101FB0541F3
:10FE8000BDF815008B894A8903449BB293428B814C
:10FE900009D3B1F800E0C0B2864540F09380897B79
:10FEA000012940F08F80122101FB0544D4F806108F
:10FEB00020881944D31A8342D8BF98B2A9F8020007
:10FEC000C9F8041016F83A3003F0400363F07703E2
:10FED00006F83830424A92F8943003F0DF0382F893
:10FEE0009430B80717D53E4C022384F8803094F83C
:10FEF000883094F88C2003A9134016208DF8143014
:10FF000000F078FABF2384F8883094F8943003F036
:10FF1000DF0384F89430F9061CD5314C202384F893
:10FF20008030102384F8803003A9142000F062FA96
:10FF300094F80C3143F0200384F80C3194F800312C
:10FF400043F0800384F8003194F8843043F02003B8
:10FF500084F88430BA060DD5214C202384F88030F3
:10FF600003A9132000F046FA94F8843003F0DF036D
:10FF700084F884303B067FF51BAF0DF10A02FF23A6
:10FF8000102103A88DF80D3000F0D0F99DF80A304B
:10FF9000134C012B04BF8DF80F3000224FF080036B
:10FFA00008BF8DF80D2003A984F88030172000F0D9
:10FFB00021FA94F8943003F0DF0384F89430F7E6E4
:10FFC000FF2210E7122202FB0544D4F80620049217
:10FFD000ADF8153003A99DF80D0000F00BFA79E794
:10FFE000002007407090FF1F5C80FF1F6BB916F860
:10FFF00032202F4902F03C02342A35D101238DF8FA
:020000021000EC
:100000000E309EF80030DB090B70122101FB054118
:100010004FF6FF734A899A42DCD0BDF815E08B8910
:1000200073449BB28B8109888E4501D19A420CD8CA
:100030008AB3B2FBF1F001FB102080B258BB122052
:1000400000FB0540807B012825D1D21A8A42D8BF07
:1000500091B2122202FB0544C9B9D4F80230C9F8A2
:100060000430A9F802102DE70A78012ACDD1FF202B
:100070000870194603A80193FFF7F4FB019B06F8EB
:1000800038301A46194603A8FFF7CAFCBDE7D4F872
:1000900006201344E3E7122202FB0544D4F80620AD
:1000A000ADF815304FF0FF330492A372E37291E77D
:1000B0005C80FF1F13460A46194601F09BB900BF3A
:1000C00030B50329039C04981DD12BB9164A226030
:1000D00004220280002030BD40F209418B420FD142
:1000E000022A4FF000030CD810490C2505FB03131E
:1000F000D9681B6951F8221021609B5C0380E9E7F5
:1001000001230122F0E7072901D9CD2030BD074B9B
:1001100003EB8102126A2260002AF6D003EB41034E
:10012000B3F84030EAE700BF5D80FF1F24170100ED
:1001300001299FBF034B5B5C1370002088BFCD205B
:10014000704700BFBC92FF1F01299DBF024B0020DA
:100150005A54CD20704700BFBC92FF1F19B14B1EEF
:1001600058425841704701207047054B1A788A421F
:1001700004D05878431A58425841704701207047BC
:10018000BC92FF1F002070470048704774170100A1
:1001900001299FBF044BC1EBC101C918002094BFC6
:1001A0001160CD20704700BF6180FF1F012930B56D
:1001B0000ED8084DC1EBC10108231068C45CC818F3
:1001C000284401330F2B00F8084CF6D1002030BD35
:1001D000CD2030BD6180FF1F01299FBF034B03EB82
:1001E00041010020116088BFCD207047BE92FF1FE3
:1001F00001299FBF034B03EB41010020116088BF21
:10020000CD207047C292FF1F01290AD813681878C1
:10021000054B03EB4101887013685B78CB700020BD
:100220007047CD20704700BFBC92FF1F01290AD83C
:1002300013681878054B03EB4101887113685B78EC
:10024000CB7100207047CD20704700BFBC92FF1FCC
:10025000084B5A7803F8022BFF210022D1540132B7
:10026000072AFBD1044A0023052199540133072BA7
:10027000FBD17047C692FF1FCF92FF1F00BF704790
:10028000013AD2B2062A10B51C4608D8054B5A705E
:10029000FFF7DEFF2146BDE81040FFF7C9B99920FE
:1002A00010BD00BFC692FF1F024B00225A70FFF71D
:1002B00031BA00BFC692FF1F37B50F4C257805B97C
:1002C000C1B98DF802308DF800109DF81830ADF8E6
:1002D000032069469DF81C2000788DF80130FFF757
:1002E00037FA9DF800301BB110B92378013B237019
:1002F00003B030BD9520FBE7C692FF1F38B50A4B0F
:100300000D461C7859788C421C4600D14DB92946BF
:100310000078FFF7D1FA2DB120B92378013323708B
:1003200038BD962038BD00BFC692FF1F4B1E062B5E
:1003300005D8094B19444B78137000207047CB0641
:1003400007D501F00F01062903D8034B19444B7A56
:10035000F2E78220704700BFC692FF1F4B1E062B9C
:100360002DE9F0418046174605D8174B19444A70CD
:100370000020BDE8F081CB0622D501F00F05062D47
:100380001ED8012A4FEAD1140F4E06D12246294623
:10039000FFF7C6FA35446F72EAE7002AFAD17319FB
:1003A0005B7A012BF6D122462946FFF789FB002D07
:1003B000F0D184F0010229464046FFF781FBE9E7CE
:1003C0008220BDE8F08100BFC692FF1F0020704769
:1003D000062903D9A1F11003072B07D8044B53F8C2
:1003E0002130002B0CBFC42000207047C420704770
:1003F0009C170100102810B50C4601D1FFF728FF0B
:10040000034B53F820300BB120469847002010BD15
:100410009C1701001FB5144602228DF807001A80B0
:1004200005210DF10F020DF10700FFF77FFF034BD0
:100430009DF80F201A80236004B010BDD892FF1FD2
:100440001FB5144601228DF807001A8004210DF112
:100450000F020DF10700FFF769FF044B9DF80F2015
:100460001A800020236004B010BD00BFD892FF1F87
:10047000F0B5002685B01E8049888DF80700ADF8DC
:100480000E10FFF76BFE18B3BDF80E20114F04AC31
:10049000B2FA82F2520901210DF10700FFF75EFF67
:1004A00034F8022D0421D2B20DF10700FFF756FFF8
:1004B0007B682246012105469DF8070098477B6826
:1004C0009DF80700324602219847284605B0F0BD46
:1004D0000425FAE7D892FF1F73B502AC002504F893
:1004E000010D0E461D80042201212046FFF736FF34
:1004F0007288024B28461A7202B070BDD892FF1F54
:1005000013B54C8889888DE80C000B46E2B2210AAD
:10051000FFF7D6FD02B010BD2DE9F04186B01746B9
:100520001E4606AA00238846059303238DF80F0074
:1005300002F8083D01210DF10F00FFF7F7FE98F8D2
:100540000050274C15F0030528D10DF111020621AA
:100550000DF10F00FFF7EAFE9DF811309DF80F0036
:1005600003F0030323800DF11203019305AB009305
:100570002A462B460221FFF7A3FD059BDB7913F0EA
:10058000400F238814BF43F0010323F001032380AD
:10059000022333803C6006B0BDE8F081012D08D114
:1005A0009DF81030012B02D198F80430ABB900232C
:1005B000EDE7022DEED198F8041041F010010DF195
:1005C0001202C9B20DF10F00FFF7B0FE9DF8123014
:1005D00003F0010323803580DCE7CD20DAE700BF9C
:1005E000D892FF1F7FB500221A800B784E788DF8C5
:1005F000070013F003030D46C6F3400634D1FEB1E5
:100600004B88013B9BB2012B52D80DF10F02062102
:100610000DF10700FFF78AFE044670B9AB7801229E
:100620009A409DF80F301A43D2B206210DF107000F
:100630008DF80F20FFF792FE0446204604B070BDEF
:100640004E88012E34D10DF10F0206210DF1070065
:10065000FFF76CFE04460028EFD1AA7896409DF87B
:100660000F2022EA0602E0E7022B21D109798DF85A
:100670000F10324641F010010DF10700FFF76EFE3A
:100680006B78002E14BF07210821012B044607D1E7
:100690009DF80F00C10900F00F00FFF7ADF9082128
:1006A000044B9DF807005B680DF10F029847C4E703
:1006B000CD24C2E7D892FF1F10B500241C800B7810
:1006C00003F00303012B05D18A780979FFF73CFD7C
:1006D000204610BD042010BD38B515460A7802F03A
:1006E0000302012A07D1054C1A8009792246FFF737
:1006F0001FFD2C6038BD042038BD00BFD892FF1FFD
:1007000013B5CD298DF8070007D1012290210DF1F5
:100710000700FFF723FE02B010BD0D491C88088AB0
:100720001268844288BF18800C461B889DF8070019
:100730000021FEF74DFF94F90A30002BEBDA00237D
:100740001A4619460DF10700FFF76AF9E3E700BF03
:10075000D892FF1F73B5054600266A4601218DF821
:1007600000600196FFF7E2FDAA78434C012A52D1BE
:1007700068680368C4F80A304368A07AC4F80E3089
:1007800004F10A0110F0600F1ED1E27A3B4B53F8DE
:100790002240002C3DD09DF80000022839D802EB01
:1007A00042021344034493F83430012B31D10DF14C
:1007B000020301AA2878A0470DF1020301AA01460D
:1007C0002878FFF79DFF13E0238AADF80230202B35
:1007D00017D87BB102060DD40A68C4F812204A6803
:1007E000C4F81620314604F11A022846FFF718F91A
:1007F00002B070BDE46B64B10DF1020301AA20499F
:10080000D8E702A82B7800F8073D9021FFF7A6FD56
:10081000EEE7CD20D0E79DF80030042B10D12B78E7
:10082000217A02AD05F8063D2846FFF7D1F90122ED
:1008300011462846FFF792FD227A03212846E5E774
:1008400094F90A30002BD3DBEB78002BD0D1E66B88
:1008500086B1B5F8093028780833ADF8023004F1D4
:1008600012010DF1020301AAB04701460DF1020386
:1008700001AAA5E7CD21F9E7D892FF1FFC170100D7
:10088000E292FF1F034B5960DA630021024AFFF72F
:100890009DBD00BFD892FF1F5507010007B502ABF1
:1008A000054A03F8010D002118465160D163FFF796
:1008B0008FFD03B05DF804FBD892FF1F0020704746
:1008C000354B41F248015A5822F00F0242F0020221
:1008D0005A5041F204015A5842F480225A5041F2CF
:1008E00034015A5842F480225A5003F52C336021C7
:1008F00093F8942042F0020283F89420C02283F8F7
:100900000021FF221A7483F8802083F8882083F85E
:100910008420002283F88C2083F80C111F491A755B
:10092000080A00F0FE0083F8982083F8C02083F8BE
:10093000C42083F8C82083F8CC2083F8D02083F823
:10094000D42083F8D82083F8DC2083F8E02083F8D3
:10095000E42083F8E82083F8EC2083F8F02083F883
:10096000F42083F8F82083F8FC2083F89C00C1F37E
:100970000740090E83F8B00083F8B41083F8AC2068
:100980001A7783F8082193F8942002F0D40242F0F9
:10099000010283F89420704700700440009CFF1F00
:1009A000024B4FF400125A60704700BF00E100E0B4
:1009B000034B4FF40012C3F884215A60704700BF04
:1009C00000E100E008B5FEF782F910B9FFF7F0FF8B
:1009D00008BD1B2008BD00BF034B4AF202629A818A
:1009E0004BF280429A81704700200540844641EADC
:1009F000000313F003036DD1403A41D351F8043B97
:100A000040F8043B51F8043B40F8043B51F8043BE8
:100A100040F8043B51F8043B40F8043B51F8043BD8
:100A200040F8043B51F8043B40F8043B51F8043BC8
:100A300040F8043B51F8043B40F8043B51F8043BB8
:100A400040F8043B51F8043B40F8043B51F8043BA8
:100A500040F8043B51F8043B40F8043B51F8043B98
:100A600040F8043B51F8043B40F8043B51F8043B88
:100A700040F8043B51F8043B40F8043B403ABDD2F7
:100A8000303211D351F8043B40F8043B51F8043B99
:100A900040F8043B51F8043B40F8043B51F8043B58
:100AA00040F8043B103AEDD20C3205D351F8043B28
:100AB00040F8043B043AF9D2043208D0D2071CBFF4
:100AC00011F8013B00F8013B01D30B88038060461D
:100AD000704700BF082A13D38B078DD010F0030393
:100AE0008AD0C3F10403D21ADB071CBF11F8013B03
:100AF00000F8013B80D331F8023B20F8023B7BE752
:100B0000043AD9D3013A11F8013B00F8013BF9D27C
:100B10000B7803704B7843708B7883706046704716
:100B200081F0004102E000BF83F0004330B54FEA9E
:100B300041044FEA430594EA050F08BF90EA020F0B
:100B40001FBF54EA000C55EA020C7FEA645C7FEA9E
:100B5000655C00F0E2804FEA5454D4EB5555B8BFC1
:100B60006D420CDD2C4480EA020281EA030382EA32
:100B7000000083EA010180EA020281EA0303362DC4
:100B800088BF30BD11F0004F4FEA01314FF4801C97
:100B90004CEA113102D0404261EB410113F0004FA9
:100BA0004FEA03334CEA133302D0524263EB430360
:100BB00094EA050F00F0A780A4F10104D5F1200EFE
:100BC0000DDB02FA0EFC22FA05F2801841F1000159
:100BD00003FA0EF2801843FA05F359410EE0A5F12D
:100BE00020050EF1200E012A03FA0EFC28BF4CF05E
:100BF000020C43FA05F3C01851EBE37101F0004514
:100C000007D54FF0000EDCF1000C7EEB00006EEB20
:100C10000101B1F5801F1BD3B1F5001F0CD34908AA
:100C20005FEA30004FEA3C0C04F101044FEA445201
:100C300012F5800F80F09A80BCF1004F08BF5FEA88
:100C4000500C50F1000041EB045141EA050130BD68
:100C50005FEA4C0C404141EB010111F4801FA4F10B
:100C60000104E9D191F0000F04BF01460020B1FA60
:100C700081F308BF2033A3F10B03B3F120020CDA98
:100C80000C3208DD02F1140CC2F10C0201FA0CF076
:100C900021FA02F10CE002F11402D8BFC2F1200CDB
:100CA00001FA02F120FA0CFCDCBF41EA0C01904091
:100CB000E41AA2BF01EB0451294330BD6FEA0404DA
:100CC0001F3C1CDA0C340EDC04F11404C4F12002C5
:100CD00020FA04F001FA02F340EA030021FA04F3D7
:100CE00045EA030130BDC4F10C04C4F1200220FA2E
:100CF00002F001FA04F340EA0300294630BD21FA6C
:100D000004F0294630BD94F0000F83F4801306BF31
:100D100081F480110134013D4EE77FEA645C18BF25
:100D20007FEA655C29D094EA050F08BF90EA020FBC
:100D300005D054EA000C04BF1946104630BD91EAB4
:100D4000030F1EBF0021002030BD5FEA545C05D1B7
:100D50004000494128BF41F0004130BD14F58004F6
:100D60003CBF01F5801130BD01F0004545F0FE416A
:100D700041F470014FF0000030BD7FEA645C1ABF9F
:100D8000194610467FEA655C1CBF0B46024650EAD6
:100D9000013406BF52EA033591EA030F41F4002102
:100DA00030BD00BF90F0000F04BF0021704730B588
:100DB0004FF4806404F132044FF000054FF000015D
:100DC00050E700BF90F0000F04BF0021704730B51E
:100DD0004FF4806404F1320410F0004548BF4042F3
:100DE0004FF000013EE700BF42004FEAE2014FEA48
:100DF00031014FEA02701FBF12F07F4393F07F4F23
:100E000081F06051704792F0000F14BF93F07F4F54
:100E1000704730B54FF4607401F0004521F0004197
:100E200020E700BF50EA010208BF704730B54FF01D
:100E300000050AE050EA010208BF704730B511F022
:100E4000004502D5404261EB41014FF4806404F15A
:100E500032045FEA915C3FF4DCAE4FF003025FEADC
:100E6000DC0C18BF03325FEADC0C18BF033202EB64
:100E7000DC02C2F1200300FA03FC20FA02F001FABE
:100E800003FE40EA0E0021FA02F11444C1E600BF5D
:100E900070B54FF0FF0C4CF4E06C1CEA11541DBF10
:100EA0001CEA135594EA0C0F95EA0C0F00F0DEF8DB
:100EB0002C4481EA030621EA4C5123EA4C5350EAC0
:100EC000013518BF52EA033541F4801143F4801311
:100ED00038D0A0FB02CE4FF00005E1FB02E506F0A2
:100EE0000042E0FB03E54FF00006E1FB03569CF0F7
:100EF000000F18BF4EF0010EA4F1FF04B6F5007FFD
:100F000064F5407404D25FEA4E0E6D4146EB06066E
:100F100042EAC62141EA55514FEAC52040EA5E50F7
:100F20004FEACE2EB4F1FD0C88BFBCF5E06F1ED8A1
:100F3000BEF1004F08BF5FEA500E50F1000041EBD8
:100F4000045170BD06F0004646EA010140EA020085
:100F500081EA0301B4EB5C04C2BFD4EB0C0541EAA7
:100F6000045170BD41F480114FF0000E013C00F3BC
:100F7000AB8014F1360FDEBF002001F0004170BDE0
:100F8000C4F10004203C35DA0C341BDC04F11404F9
:100F9000C4F1200500FA05F320FA04F001FA05F285
:100FA00040EA020001F0004221F0004110EBD37052
:100FB00021FA04F642EB06015EEA430E08BF20EA7E
:100FC000D37070BDC4F10C04C4F1200500FA04F321
:100FD00020FA05F001FA04F240EA020001F00041B3
:100FE00010EBD37041F100015EEA430E08BF20EA26
:100FF000D37070BDC4F1200500FA05F24EEA020E6E
:1010000020FA04F301FA05F243EA020321FA04F09C
:1010100001F0004121FA04F220EA020000EBD37053
:101020005EEA430E08BF20EAD37070BD94F0000F53
:101030000FD101F00046400041EB010111F4801F87
:1010400008BF013CF7D041EA060195F0000F18BF38
:10105000704703F00046520043EB030313F4801F74
:1010600008BF013DF7D043EA0603704794EA0C0F2E
:101070000CEA135518BF95EA0C0F0CD050EA410644
:1010800018BF52EA4306D1D181EA030101F00041C1
:101090004FF0000070BD50EA410606BF10461946E9
:1010A00052EA430619D094EA0C0F02D150EA0136F5
:1010B00013D195EA0C0F05D152EA03361CBF104636
:1010C00019460AD181EA030101F0004141F0FE41D5
:1010D00041F470014FF0000070BD41F0FE4141F459
:1010E000780170BD70B54FF0FF0C4CF4E06C1CEA59
:1010F00011541DBF1CEA135594EA0C0F95EA0C0F0E
:1011000000F0A7F8A4EB050481EA030E52EA0335C8
:101110004FEA013100F088804FEA03334FF08055E9
:1011200045EA131343EA12634FEA022245EA111516
:1011300045EA10654FEA00260EF000419D4208BFC7
:10114000964244F1FD0404F5407402D25B084FEA74
:101150003202B61A65EB03055B084FEA32024FF420
:1011600080104FF4002CB6EB020E75EB030E22BF7D
:10117000B61A754640EA0C005B084FEA3202B6EB3D
:10118000020E75EB030E22BFB61A754640EA5C00EC
:101190005B084FEA3202B6EB020E75EB030E22BF7C
:1011A000B61A754640EA9C005B084FEA3202B6EB7D
:1011B000020E75EB030E22BFB61A754640EADC003C
:1011C00055EA060E18D04FEA051545EA16754FEA9E
:1011D00006164FEAC30343EA52734FEAC2025FEABC
:1011E0001C1CC0D111F4801F0BD141EA00014FF04B
:1011F00000004FF0004CB6E711F4801F04BF01431C
:101200000020B4F1FD0C88BFBCF5E06F3FF6AFAE37
:10121000B5EB030C04BFB6EB020C5FEA500C50F1C7
:10122000000041EB045170BD0EF0004E4EEA11314A
:1012300014EB5C04C2BFD4EB0C0541EA045170BD51
:1012400041F480114FF0000E013C90E645EA060E95
:101250008DE60CEA135594EA0C0F08BF95EA0C0FC3
:101260003FF43BAF94EA0C0F0AD150EA01347FF40B
:1012700034AF95EA0C0F7FF425AF104619462CE7E2
:1012800095EA0C0F06D152EA03353FF4FDAE104645
:10129000194622E750EA410618BF52EA43067FF496
:1012A000C5AE50EA41047FF40DAF52EA43057FF426
:1012B000EBAE12E74FEA410212F5001215D211D53A
:1012C0006FF47873B3EB625212D94FEAC12343F043
:1012D000004343EA505311F0004F23FA02F018BFC5
:1012E000404270474FF00000704750EA013005D18E
:1012F00011F0004008BF6FF0004070474FF0000051
:10130000704700BFFDF7ABFB002103E00A4B5B58C1
:101310004350043109480A4B42189A42F6D3094A0D
:1013200002E0002313600432074B9A42F9D300F025
:101330000DF8804770470000881801000880FF1FE3
:101340007485FF1F0086FF1F24A0FF1F264C08B5D1
:10135000F7F797F8F7F7FEF8F7F764FAF7F776FA82
:10136000F7F780F9F7F75AFCFCF716FCFCF7FEF9E3
:10137000F7F7C0FDF7F70CFB2078F7F783F9E07873
:10138000F7F7F0F9F7F7ADFB28B1F7F7AAFB6070B4
:10139000F7F7A7FBA060F7F71DFC21896079228A87
:1013A000FCF73EFAFDF752FAFDF7FAF8FCF78AFC73
:1013B0000E4B4FF400725A60F8F744FCFBF708FB41
:1013C0000B4B04225A60FAF75FFFFBF7DFFBFBF7DA
:1013D00000FBF7F7BAFBF7F7EDFB0028F3D0FDF7BA
:1013E000DFF8F8F72FFCEEE70C80FF1F80F00F40CE
:1013F00000F00F4070B4860746D0541E002A41D03A
:10140000CAB2034602E014F1FF343BD303F8012BC8
:101410009D07F8D1032C2ED9CDB245EA05250F2C16
:1014200045EA054519D903F110022646103E0F2E54
:1014300042F8105C42F80C5C42F8085C42F8045C2C
:1014400002F11002F2D8A4F1100222F00F0204F00F
:101450000F041032032C13440DD91E462246043AC1
:10146000032A46F8045BFAD8221F22F00302043252
:10147000134404F003042CB1C9B21C4403F8011B4B
:101480009C42FBD170BC704714460346C2E700BFC4
:10149000024B13B1024800F005B87047000000008D
:1014A000B1140100002301461A46184600F01EB888
:1014B00038B50A4C0A4D641BA4100AD004F18043CD
:1014C000013B05EB8305013C55F804399847002C96
:1014D000F9D1BDE8384000F0CBB900BF8818010051
:1014E00084180100704700BF704700BF2DE9F84322
:1014F0002C4D0646286898460F469146FFF7F2FFA6
:10150000294B1C68D4F84831002B3ED05A681F2A5A
:101510001CDC02F1010E76B103EB82010124C1F85B
:101520008890D3F8880194402043022EC3F88801A4
:10153000C1F8088123D00232C3F804E0286843F8D8
:101540002270FFF7D1FF0020BDE8F883174B0BB3E3
:101550004FF4C870AFF300800346D8B1D4F84821E7
:101560000260002141600A46C4F848014FF0010EB4
:10157000C0F88811C0F88C11002EDCD0CCE7D3F86D
:101580008C110C43C3F88C41D5E704F5A673C4F85D
:101590004831BBE72868FFF7A7FF4FF0FF30BDE8F1
:1015A000F88300BF7085FF1F601801000000000075
:1015B0008025000040380000004B000080700000D3
:1015C0000096000000E10000002C010000C20100B4
:1015D0000084030090D0030020A1070040420F00C8
:1015E00000000000E0930400C0270900FF00000194
:1015F0000000000064F00000E80300001027000075
:1016000010270000140000000A0000000000000085
:10161000FFFFFF3F000001006400000064000000C5
:1016200000070000F40100000000000000000000BE
:1016300000000000000000000000000000000000AA
:101640000050C3000088130001400808000000009B
:1016500000000000C8000000010000000080000041
:1016600000000000000000000000C800002003008F
:10167000000000000000000000000000C8000000A2
:10168000000000000000000000000000000000005A
:10169000000000000000000000000000000000004A
:1016A0000000000001010100010000000000000036
:1016B0000000000000000100000000000000000029
:1016C0000000000001010100000000000000000017
:1016D0000001000000000000010101000101000103
:1016E00001000000000000000000000000000000F9
:1016F00000000000000000000000000000000000EA
:1017000000000000000000000000000000000101D7
:1017100001000001000100010000000000000000C5
:10172000000000005D80FF1F0400000009040000AD
:101730008817010098170100000000000000000059
:1017400000000000000000003481FF1FF180FF1F37
:101750000000000000000000000000000000000089
:101760000000000000001200430000000000000024
:10177000000000000301020110000202001000033B
:1017800003011000000100005D80FF1FB780FF1FF4
:101790009180FF1F6F80FF1F043A2622550701002A
:1017A00051F00000E9F0000059EE00007D02010058
:1017B0007D0201007D0201007D0201007D02010029
:1017C0007D0201007D0201007D0201007D02010019
:1017D0007D0201007D0201007D020100DBF30000BB
:1017E00071F30000D1F300009DF3000071F30000DD
:1017F0007D0201005DF3000049F4000019050100BD
:10180000E505010000000000E50501000000000002
:10181000D90401000105010000000000410401009D
:1018200071040100D9060100B90601001504010088
:1018300001010001010000000001010000000000A2
:10184000010101010100000001010001010001008E
:1018500000010000010000333331325631303700CF
:101860004881FF1FF8B500BFF8BC08BC9E46704712
:0C187000F8B500BFF8BC08BC9E467047ED
:08187C00911401003584000005
:0418840011840000CB
:1018880057180100000102000008000001000000D4
:10189800020000000000000000000000000000003E
:1018A8000000000000000000000000000000000030
:1018B8000000000000000000000000000000000020
:1018C80000000000010002000400A1200000000048
:1018D80002000000FF0403090400C2010000000820
:1018E80000000000000000220342004100440020E4
:1018F8000053005400520049004E004700200049A0
:10190800004E00440045005800260353007400654B
:1019180000700070006500720020004D006F0074B8
:10192800006F007200200044006500760020003A35
:10193800035400520049004E0041004D0049004345
:101948000020004D006F00740069006F006E0020D9
:101958000043006F006E00740072006F006C00207E
:10196800002000200020002000090243000201009E
:10197800C032090400000102020000052400100121
:1019880005240101010424020605240600010705B7
:10199800830310000A09040100020A000000070579
:1019A8008102100000070502021000001201000267
:1019B800020000103C2A00010200010200010000A0
:1019C800000000003484FF1F9C84FF1F0485FF1F54
:1019D80000000000000000000000000000000000FF
:1019E80000000000000000000000000000000000EF
:1019F80000000000000000000000000000000000DF
:101A080000000000000000000000000000000000CE
:101A180000000000000000000000000000000000BE
:101A280000000000000000000000000000000000AE
:101A3800000000000000000000000000000000009E
:101A4800000000000000000000000000000000008E
:101A5800000000000000000000000000000000007E
:101A6800000000000000000001000000000000006D
:101A78000E33CDAB34126DE6ECDE05000B00000032
:101A8800000000000000000000000000000000004E
:101A9800000000000000000000000000000000003E
:101AA800000000000000000000000000000000002E
:101AB800000000000000000000000000000000001E
:0C1DE800000000000000000000A0FF1F31
:101DF400881801000880FF1F6C0500000000000027
:081E04000000000000000000D6
:020000020000FC
:020000041FFFDC
:04800000000000007C
:0400000310001305D1
:00000001FF
